:04000005000080C1B6
:020000040000FA
:10800000102300200983000011830000FD9500006B
:10801000000000000000000000000000D940FEDF6A
:108020008F9E939B01999697FA000000B9810000FA
:1080300000000000000000005D820000BD82000022
:108040001B8300001B8300001B8300001B830000B8
:108050001B8300001B8300001B8300001B830000A8
:108060001B8300001B8300001B8300001B83000098
:108070001B830000D19C00001B8300001B830000B9
:108080001B8300001B8300001B8300001B83000078
:108090001B8300001B8300001B8300001B83000068
:1080A000B99D00001B8300001B8300001B830000A0
:1080B0001B8300001B8300001B8300001B83000048
:1080C00000F002F800F030F80CA030C8083824188E
:1080D0002D18A246671EAB4654465D46AC4201D100
:1080E00000F022F87E460F3E0FCCB6460126334202
:1080F00000D0FB1AA246AB463343184724AF00001A
:1081000044AF00000023002400250026103A01D3CC
:1081100078C1FBD8520700D330C100D50B6070473F
:108120001FB51FBD10B510BD00F076FB1146FFF75F
:10813000F7FF05F0C3FE00F08EFB03B4FFF7F2FF7C
:1081400003BC00F03FFB000080F309887047EFF3A9
:1081500009807047684680F3098806480078C007A0
:1081600003D1032080F314887047022080F3148821
:1081700070470000F81E0100064B9C46EFF3058394
:108180001B0605D1EFF31483DB0701D000DF704736
:108190006047000005EB0000064B9C46EFF30583AB
:1081A0001B0605D1EFF31483DB0701D000DF704716
:1081B0006047000019ED0000EFF309808169891E16
:1081C0000978002933D1A6461FC8A4467446E04763
:1081D0001F4B06CB914224D0083B002910D00CB491
:1081E000203101234B70EFF30983203B4B60F0C338
:1081F00044464D4656465F46F0C307F023F80CBC94
:108200001A60203253681033F0CBA046A946B2461C
:10821000BB4683F30988203BF0CB5078002803D07D
:108220001078EFF3098318600223DB43184710B579
:10823000084A1268914209D8074C89006458A6463A
:108240001FC8A446F047EFF309840FC410BD000017
:10825000A0F1FF1FFC880000FC88000006F0D8FE9B
:10826000154B06CB914223D0083B0CB420310023A0
:108270004B70EFF30983203B4B60F0C344464D46FF
:1082800056465F46F0C306F0DDFF0CBC1A60203294
:1082900053681033F0CBA046A946B246BB4683F3E1
:1082A0000988203BF0CB5078002801D01078186165
:1082B0000223DB4318470000A0F1FF1F07F07AF804
:1082C000CEE7000005F0CCFF07F074F8C8E7000027
:1082D00070B505460C46164602E00FCC0FC5103EA1
:1082E000102EFAD2082E02D303CC03C5083E042E6A
:1082F00007D301CC01C5361F03E021782970641C27
:108300006D1C761EF9D270BD0748804707480047AC
:10831000FEE7FEE7FEE7FEE7FEE7FEE70448054965
:10832000054A064B70470000219C0000C1800000F8
:1083300010210020102300201022002010220020F5
:1083400000487047AC20002010B5002000F040FA33
:10835000FFF7E8FE012000F035FA10BD034610B526
:108360000B439B070FD1042A0DD308C810C9121F55
:10837000A342F8D018BA21BA884201D9012010BD11
:108380000020C04310BD002A03D0D30703D0521CE5
:1083900007E0002010BD03780C78401C491C1B1B13
:1083A00007D103780C78401C491C1B1B01D1921E7D
:1083B000F1D1184610BD000030B5441C03E001782F
:1083C000401C00290DD08107F9D10B4BDD0104C8F9
:1083D000D11A91432940FAD0001B0A0603D0C01ECF
:1083E00030BD001B30BD0A0401D0801E30BD090223
:1083F000FCD0401E30BD00000101010170477047F4
:10840000FFFFFFFFFFFFFFFFFFFFFFFFFEFFFFFF7D
:108410000346F0B50B439B072DD1244DEF01042AF1
:1084200029D308C810C95E1B9E43121F3E4017D0B7
:10843000D8B2E1B2401A3106014310D198B2A1B2CC
:10844000401A310401430AD118022102000A090A24
:10845000401A3102014302D1180E210E401AF0BD1C
:10846000A342DCD018BA21BA884201D90120F0BD5C
:108470000020C043F0BD002A01D10020F0BD0378E8
:108480000C78401C491C002B0DD0A3420BD1521E6E
:1084900009D003780C78401C491C002B03D0A34260
:1084A00001D1521EEBD1181BF0BD000001010101EA
:1084B000421E5378521C002BFBD10B78491C1370C1
:1084C000521C002BF9D17047F8B5042A2CD383072E
:1084D00012D00B78491C0370401C521E83070BD02E
:1084E0000B78491C0370401C521E830704D00B7884
:1084F000491C0370401C521E8B079B0F05D0C91AE4
:10850000DF002023DE1B08C90AE0FFF7E1FEF8BD0B
:108510001D4608C9FD401C46B4402C4310C0121F24
:10852000042AF5D2F308C91A521EF0D40B78491C5C
:108530000370401C521EEAD40B78491C0370401C87
:10854000012AE4D409780170F8BD431A70B593424A
:108550001BD28918801804E0491E401E0B78521E59
:1085600003709307F8D106E01039103878C9103934
:1085700078C01038103A102AF6D203E0091F001F05
:108580000B680360121FF9D570BDFFF7A1FE70BD27
:10859000F8B5064614460843800707D0751AA54269
:1085A00019D20819102D13D2311907E03046FFF700
:1085B000CCFFF8BD401E491E02780A70641EF9D235
:1085C000F8BD471B2A463946FFF77EFF641B384635
:1085D000A542F6D3011B22463046FFF775FFF8BDD2
:1085E000D2B210B513029A1813049A1800F00EF8BC
:1085F00010BD01E004C0091F0429FBD28B0701D57F
:108600000280801CC90700D00270704700290BD07F
:10861000C30702D00270401C491E022904D38307FD
:1086200002D50280801C891EE3E70022EEE70022CB
:10863000DFE70378C2781946437812061B02194314
:108640008378C0781B04194311430902090A000604
:1086500008437047020A08704A70020C8A70020EC2
:10866000CA707047002203098B422CD3030A8B4245
:1086700011D300239C464EE003460B433CD400221A
:1086800043088B4231D303098B421CD3030A8B422C
:1086900001D394463FE0C3098B4201D3CB01C01AFA
:1086A000524183098B4201D38B01C01A52414309C5
:1086B0008B4201D34B01C01A524103098B4201D3B3
:1086C0000B01C01A5241C3088B4201D3CB00C01A20
:1086D000524183088B4201D38B00C01A5241430898
:1086E0008B4201D34B00C01A5241411A00D20146BD
:1086F0005241104670475DE0CA0F00D04942031056
:1087000000D34042534000229C4603098B422DD3A4
:10871000030A8B4212D3FC22890112BA030A8B424C
:108720000CD3890192118B4208D3890192118B429B
:1087300004D389013AD0921100E08909C3098B4220
:1087400001D3CB01C01A524183098B4201D38B0163
:10875000C01A524143098B4201D34B01C01A524106
:1087600003098B4201D30B01C01A5241C3088B424B
:1087700001D3CB00C01A524183088B4201D38B0036
:10878000C01A5241D9D243088B4201D34B00C01AC0
:108790005241411A00D20146634652415B101046D5
:1087A00001D34042002B00D54942704763465B101D
:1087B00000D3404201B50020C046C04602BD70470C
:1087C0007047704701491820ABBEFEE72600020043
:1087D00010B500F009F800F001F810BD10B5002840
:1087E00001D0FFF7EFFF10BD10B5002102A000F08F
:1087F0003AF8012010BD0000534947414252543A13
:108800002041626E6F726D616C207465726D696E6D
:108810006174696F6E0000007546FFF791FDAE460A
:10882000050069465346C008C000854618B020B50B
:10883000FFF774FD60BC00274908B6460026C0C596
:10884000C0C5C0C5C0C5C0C5C0C5C0C5C0C5403D08
:1088500049008D46704710B50446C046C0462046C4
:10886000FFF76BFC10BD70B505460C460A2000E012
:108870006D1C00F012F8002D06D028780028F7D1E2
:1088800002E0641C00F009F8002C02D020780028D7
:10889000F7D10A2000F001F870BD08B569460870EC
:1088A0000320ABBE08BD70B58C180578401C6B0763
:1088B0005B0F01D10378401C2A1106D10278401CBD
:1088C00003E00678401C0E70491C5B1EF9D12B0793
:1088D00005D40023521E0DD40B70491CFAE703780F
:1088E000401CCB1A921C03E01D780D70491C5B1CC8
:1088F000521EF9D5A142D8D3002070BD000000005F
:10890000F8B502787F2A02D000F018F8F8BD0A7096
:108910004478861C4C708D1C074F08E02946304671
:1089200000F00CF8010C3F188E1980B24519641E36
:10893000F4D23846F8BD000002000200F8B5027813
:108940001346803B1F2B02D800F036F9F8BD0A70A1
:1089500007784C1C421C0025FF219048904E3B009C
:1089600003F030FE170D37405DB7C4E1F2F16E77CA
:10897000F2F2F2F2F27B8085949EB45AF200117802
:10898000601C0022062920D006DC0B0003F01AFE32
:10899000051D1D1D1D0D1D00F0290CD0FD2914D035
:1089A000FE290FD0FF2910D107E005227D49FFF7EE
:1089B0008BFD052209E0112105E040210170457081
:1089C000022202E00521017001227748227010186E
:1089D000F8BD107800283AD0012838D021707248AC
:1089E000401EC4E01178002903D0012902D00021E3
:1089F00012E00121012202706C48202343604025CF
:108A000045608215426047691F43476143692B43B4
:108A1000436143691343436121703046A7E0057009
:108A20006248426920218A434261426940218A4367
:108A30004261426981158A4342612570012096E0B6
:108A400050781178000208430001401EFDD12570C6
:108A5000C5E765702570022089E02146104600F0C8
:108A600085FB84E02146104600F050FB7FE017783C
:108A7000511C002F01D1FF270137384601F0AAF819
:108A8000FF1D2570F8080004801970E011788A072E
:108A9000920F521C49070275C90F41752570BCE73A
:108AA0002170012113780C46521C0AE01078521CE8
:108AB0008006800E00D14020C01DC0081218091881
:108AC000491C5B1EF2D20804204350E0107821704C
:108AD000D9E71178017293785778190239434181A7
:108AE0001179D27809021143818150E00078214642
:108AF000012814D01346521C1078521C002808D0AC
:108B00001778521CBC0701D5FC0600D5121D401E6B
:108B1000F6D1D01A0D7000044D70801C27E010466D
:108B200000F0D0F823E000781746214601280CD049
:108B30000D704D70A5700320F9781D4A890708D57E
:108B4000104301460CE00DE023E0104600F04CFA23
:108B5000F2E7B9787B78090219438904891801433F
:108B6000084604E00078012803D0217011488019DC
:108B7000F8BD1746501CFFF75CFD39790002000A6A
:108B80000906084300906946002000F0B1FD2570F9
:108B9000ECE7203CE1773046F8BD0000A8F2FF1F6B
:108BA000010001004C1E01000200020080F00F4095
:108BB0000000040001000500FEB502780A704D1C9B
:108BC00001783D4C401C80390646671C0B0003F0C1
:108BD000F9FC0D08162238407171714755606468C0
:108BE000710004F0EBFF0746FFF7E6FBC6B22E70FC
:108BF000681C32463946FFF767FCA41927E00724B2
:108C0000684601F0ABFA224669462846FFF75CFC4D
:108C1000294C08344EE0684601F0A0FA002002908A
:108C20000422314602A8FFF74FFC029800906846E4
:108C300001F0B4FA002001F031FB012028701F4C34
:108C400038E03E21681C07F0EBFD28702418641CF6
:108C500030E03778401C394607F050FE012025E00F
:108C6000012028703078002805D0012803D000208A
:108C70002870134C1EE005F09BFAFAE701202870DB
:108C800003F098FE002802D1022007F085FB3C4645
:108C900010E0007806F052FDEAE706F01BFD2870B0
:108CA000F5E73778401C394606F0F0FD28703904A6
:108CB000081904192046FEBD01000100020005004C
:108CC00002000200F0B589B00890044600208D1C17
:108CD0000391C34902900870049005906678A41C23
:108CE000002E6FD02778641CB9076CD50499002931
:108CF00035D0BC48408901901120384001280FD15F
:108D00006946384600F0F4FC02281AD10199491E40
:108D10000191491C03D0B24909780029F0D012E131
:108D200069460E2000F0E4FC022808D10199491E92
:108D30000191491C03D0AA4909780029F0D00021EB
:108D400004910128EBD1009929700099090A6970F2
:108D50000099090CA9700099090EE9702D1DF906FA
:108D600058D52046FFF765FCE1780002000A0906A5
:108D7000084307909B48241D80890690F80715D06A
:108D80009848408901900021384600F0B1FC022843
:108D900002D00128C3D109E00199491E0191491C63
:108DA000BDD08F4909780029EDD0CCE08D484089AD
:108DB00001906946384600F09BFC022804D0012847
:108DC0001CD10BE0E0E064E00199491E0191491CCF
:108DD00014D0834909780029EBD00FE08149009A2B
:108DE00009691140079A914208D00699491E0691D7
:108DF000491C03D07A4909780029D7D07949009ACB
:108E000009691140079A914201D0102108430128B5
:108E10001AD13CE0734949890191F90718D00499A6
:108E2000002934D10021384600F062FC022802D02B
:108E3000012809D109E00199491E0191491C03D07B
:108E4000674909780029EDD07DE0012104911EE0F9
:108E50006946384600F04CFC022802D0012872D145
:108E600009E00199491E0191491C6CD05C490978BF
:108E70000029EDD067E0009929700099090A69700E
:108E80000099090CA9700099090EE9702D1D0021A7
:108E90004DE00498002823D052484089019069464B
:108EA0000E2000F025FC022802D001284BD109E059
:108EB0000199491E0191491C45D049490978002969
:108EC000EDD040E0009828700098000A6870009883
:108ED000000CA8700098000EE87000202D1D049072
:108EE0002046FFF7A6FBE1780002000A09060843C6
:108EF000241D0090B90603D53A490861012017E006
:108F00003848408901906946384600F0F1FB022854
:108F100002D0012817D109E00199491E0191491C8D
:108F200011D02F4909780029EDD00CE001210591DD
:108F30000299491C02912A490978002903D1761E19
:108F400000D0CFE60AE0002E08D02178641C8A0702
:108F500001D5C90600D5241D761EF4E7012832D1BB
:108F6000049900291ED01F481D4F468969460E20CE
:108F700000F0BEFB022802D0012824D105E0761EB5
:108F800021D339780029F1D01DE00099297000998A
:108F9000090A69700099090CA9700099090EE97015
:108FA0002D1D10E0059900290DD00E480C4F468963
:108FB00000210E2000F09CFB022804D1761E02D373
:108FC00039780029F4D0039A0299117003994870F6
:108FD00008980399201A0004691A084309B0F0BDE3
:108FE00004F0FF1FA8F2FF1FF3B583B00025CE1CCD
:108FF00002914449024628460D70917853780C023C
:10900000D21C1C4373D01178521C00910392890723
:109010005DD50099C90737D03B48478900210098A2
:1090200000F066FB022802D0012860D12CE07F1EF0
:109030005DD3344909780029F0D058E0002C04D1E0
:109040000098C00701D00E2000902F48478901A941
:10905000009800F04DFB022802D0012847D106E01D
:109060007F1E44D3274909780029F0D03FE00199B9
:10907000317001996D1C090A71700199090CB17068
:109080000199090EF170361D641ED7D22FE00398A6
:10909000FFF7CFFA03990002C978000A09060843CE
:1090A00001900398001D03901748478901A9009873
:1090B00000F01EFB022802D0012818D106E07F1E16
:1090C00015D3104909780029F0D010E06D1C641EFA
:1090D000DDD20D480B4F448900210E2000F008FB23
:1090E000022804D1641E02D339780029F4D00299F1
:1090F0000D70029A290A517002998870029805B081
:10910000301AF0BD04F0FF1FA8F2FF1FF8B50C469F
:109110000546FFF78EFA0102E878090A0006104FAB
:10912000014307D00F4800260F4D814205D301208F
:10913000687010E0FF2020700FE00A486E70401E3B
:109140000818FFF78FFA012804D90321401CFFF704
:1091500089FA00E00120686026703846F8BD0000FA
:109160000100040000366E01A8F2FF1FF8B50746A3
:10917000057844780E46801CFFF75BFA0102787987
:10918000090A000601432F48E20706D0EB07202218
:10919000002B01D0426000E08260A20706D5AB0739
:1091A0004022002B01DA426000E08260220606D5F0
:1091B000EA09D307244A01D0426000E0826000231C
:1091C00000292ED0214A914200D91146204A9361AC
:1091D00030277943516105211161E10704D001690C
:1091E0008906C90FA94217D1A10705D501696F08E2
:1091F0004906C90FB9420FD1610701D5A9080BD1A2
:10920000A10601D5690907D1210609D50169EF0930
:10921000C905C90FB94203D01169C903C90FDCD010
:109220001361016902698906C90F5206D20F520003
:1092300000691143C005C00FC001014331700548EA
:10924000F8BD000080F00F4000010000C0C62D00F6
:1092500000E000E00100060010B516480021017092
:1092600041700322426001726422428181810122A5
:109270000161027541751048816B1F225202114332
:109280008163FF200D49033048610D482022426070
:10929000436913434361FF2404348C6140224260DC
:1092A0004369934343610C628115416042690A43FB
:1092B000426110BDA8F2FF1F0080044000B00440CE
:1092C00080F00F4070B50546EFF31080C407E40F3F
:1092D00072B6094E094B29463046F26800F010F884
:1092E000002805D1002329463046F26800F000F935
:1092F000002C00D162B670BD0C1300206B66656B4C
:10930000FFB589B016460C466A46099804F0D2F9B2
:1093100032462146049B099803F08FFF05002BD1AC
:10932000009C019FA619761E39463046FFF79AF930
:1093300000291BD0401C7843461E17E0210209205B
:10934000090A000609180D4841600C9803F08EFFC9
:10935000002811D1099803F093FF05460998006988
:10936000002800D08047002D02D1E419B442E5D98D
:10937000099803F035FF28460DB0F0BD000002400B
:1093800070B5040027D01648C0680001000F0F28F0
:1093900023D014494000085A8002002525606060EF
:1093A0000120A0606561A56180022561E060204622
:1093B00003F035FF00280AD00B48014680390560CC
:1093C000416040318160E061204600F00FF8256285
:1093D0000020656270BD042070BD01204004DCE700
:1093E0004080044020230100C013002070B50028F5
:1093F00022D0C46916484022410816484900400856
:1094000040006568884202D9421A402A12D828468C
:10941000FFF75AF81148104E410811486D1C35608D
:109420004008402249004000A568884206D9421AF7
:10943000402A03D9FEF788FF042070BD2846FFF7B5
:1094400043F86D1C022075602060002070BD000094
:1094500095D90000A1D9000020F1FF1F09D200001A
:109460001DD20000FFB589B01F4614000D460DD077
:109470006A46099804F01EF93A462946039B099862
:1094800003F0DBFE060002D1009D28E004200DB0B1
:10949000F0BD02CC154881600399042902D0082947
:1094A00007D00EE029020322090A520689184160FA
:1094B00007E002CCC16029020722090A12068918B6
:1094C0004160099803F0DCFE06460998006900280F
:1094D00000D08047002E04D1039845193F1A002F71
:1094E000D7D1099803F07CFE3046D0E70000024057
:1094F000FFB589B014460D466A46099804F0DAF8BB
:1095000022462946059B099803F097FE00282FD193
:109510006A462946099804F0CDF8009D0298089003
:109520006942404201404F42AF4201D108983F1882
:10953000002C1CD07E1BA64200D926463046059939
:10954000FFF790F829020122090A12068A18094930
:109550004A600C9A000412021043FF308860099898
:1095600003F08EFE002803D1A41BAD19DEE7002016
:109570000DB0F0BD00000240FFB589B0129F1D0084
:1095800016460C4610D06A46099804F093F8324605
:109590002146079B099803F050FE002805D1154A83
:1095A00039068F18009C22E004200DB0F0BD210286
:1095B0000120090A400609180F48416087602968A0
:1095C000C160099803F05CFE002809D013990029B6
:1095D00000D00C6014990029E7D000220A60E4E76B
:1095E0000799761A890889004D1907990C19002ED8
:1095F000DDD1DAE7FFFFFF0000000240BA2203A13D
:10960000002003F02FF800F057FBFEE72E2E5C2E13
:109610002E5C2E2E5C736F757263655C6461706C7A
:10962000696E6B5C696E746572666163655C6D61C1
:10963000696E2E630000000010B5EFF31080C007C4
:10964000C00F72B60021064A1160002800D162B630
:109650000448FFF795FE002800D0012010BD00004F
:10966000008104400C1300201CB506F011FB0028FB
:109670001AD09E2069460870E7204870102000F03C
:10968000A9FA012406F004FB00280DD00020694649
:109690000870082000F09EFA01A9002006F08EFA5A
:1096A000012802D1002C00D01CBD00201CBD0000F0
:1096B000FEB5074616460D46EFF31080C407E40FCB
:1096C00072B60B4639460948FFF7CCFE002809D18F
:1096D000012101900091029033462A463946034801
:1096E000FFF74AFF002C00D162B6FEBD0C1300202C
:1096F00000B5054A5278002A02D000F007F800BDF4
:1097000000F0E0F800BD0000A8F2FF1FF0B58C46A5
:109710006A4E4021024671602027B7607760C0071B
:1097200001D0716000E0B160B76077605008C40795
:1097300001D0716000E0B160B760776013189008E5
:10974000C40701D0716000E0B160B76077601B189A
:10975000D008C40701D0716000E0B160B7607760E5
:109760001818C00701D0716000E0B160B760776081
:10977000B160B76077607160B76077607069884387
:1097800070614F48007D041E03D0B7607760401EB3
:10979000FBD1B760306977604006C00FB7603369AE
:1097A00077605B06DB0F5B000343B760306977606F
:1097B0004006C00F8000184301280DD002285DD05C
:1097C00004285BD0213403D0B7607760641EFBD1DE
:1097D00072690A4372616FE0920726D500231C4626
:1097E0002022B760356977606D06ED0F64195B085C
:1097F000ED072B43521EF4D1B760326977605206F1
:10980000D20F5440E20700D008206246002A00D060
:1098100013602B4A127D002A03D0B7607760521E76
:10982000FBD172690A4372611EE0002C03D0B7605D
:109830007760641EF9E772690A43726162461268D2
:1098400000242023D50701D0716000E0B160B7602B
:109850007760A41852085B1EF4D1E20701D0716052
:1098600000E0B160B7607760154A127A002A23D011
:10987000B160B7607760521EFBD11DE0104B5D7D7B
:10988000002D06D0930704D52123B76077605B1EB7
:10989000FBD1002C03D0B7607760641EF9E77369D1
:1098A0000B437361002D07D0920705D4B1602122CC
:1098B000B7607760521EFBD17160F0BD80F00F4041
:1098C000A8F2FF1FF0B503460022C04D40208C4691
:1098D00068602024AC60BE4F79680E46761EFDD1CC
:1098E0006C600E46761EFDD1DE0701D0686000E098
:1098F000A860AC600E46761EFDD16C600E46761EEA
:10990000FDD1D6185A08D70701D0686000E0A860DA
:10991000AC600F467F1EFDD16C600F467F1EFDD1EF
:10992000B6189A08D70701D0686000E0A860AC605C
:109930000F467F1EFDD16C600F467F1EFDD1B6180D
:10994000DA08D70701D0686000E0A860AC600F4675
:109950007F1EFDD16C600F467F1EFDD1B218D2076D
:1099600001D0686000E0A860AC60994E0A46521EC3
:10997000FDD16C600A46521EFDD1A860AC600A465B
:10998000521EFDD16C600A46521EFDD16860AC606B
:109990000A46521EFDD16C600A46521EFDD16A690C
:1099A000402082436A61327D161E09D0AC600846B1
:1099B000401EFDD16C600846401EFDD1521EF5D1FF
:1099C000AC600846401EFDD128696C604006C00F9F
:1099D0000A46521EFDD1AC600A46521EFDD12A69CC
:1099E0006C605206D20F0F467F1EFDD1520002431B
:1099F000AC600846401EFDD128694006C70F2020F4
:109A000068600846401EFDD1B8001043012816D0FA
:109A100002286ED004286CD021360AD02023AB60F7
:109A20000A46521EFDD16B600A46521EFDD1761EBB
:109A3000F5D169694022114369616A60F0BD9A07F6
:109A40003CD50024264620232027AF600A46521E1C
:109A5000FDD12A696F605206D20F0F467F1EFDD1DD
:109A60006708D407B6183C435B1EEDD120232A4675
:109A7000AB600F467F1EFDD1176953607F06FF0F55
:109A8000491EFDD17E40F10700D008206146002923
:109A900000D00C604E490C7D002C0AD04E689360BB
:109AA0003146491EFDD153603146491EFDD1641E29
:109AB000F5D1516940231943516139E0002E0AD094
:109AC0002023AB600A46521EFDD16B600A46521E2F
:109AD000FDD1761EF5D16A6940231A436A61624658
:109AE0000026126820242746D30703D040236B604A
:109AF00002E032E04023AB60AF600B465B1EFDD15D
:109B00006F600B465B1EFDD1B6185208641EEBD188
:109B1000F20702D040226A6001E04022AA603B4680
:109B20002C46AF600A46521EFDD16360491EFDD12E
:109B300027490A7A002A0DD04023AB604B682024C5
:109B4000AC601946491EFDD16C601946491EFDD115
:109B5000521EF5D140216960F0BD1D4A527D9446E8
:109B6000002A0DD09A070BD521242027AF600A4682
:109B7000521EFDD16F600A46521EFDD1641EF5D102
:109B8000002E0AD02024AC600A46521EFDD16C6023
:109B90000A46521EFDD1761EF5D16A694024224341
:109BA0006A616246002A0ED09A070CD4AC60212369
:109BB0002026AE600A46521EFDD16E600A46521E35
:109BC000FDD15B1EF5D16C60F0BD000080F00F4050
:109BD000A8F2FF1FF0B50023104C1A460E4E2027A6
:109BE000656815E0002A02D10B780822491CDC07C1
:109BF00002D04024746001E04024B460B7602C4679
:109C0000641EFDD177602C46641EFDD15B08521E98
:109C1000401EE7D2F0BD000080F00F40A8F2FF1F09
:109C20001E48002202601E48816B43151943816360
:109C30001B491C48403148601B4883681B490B4046
:109C40008360C3680B40C3601949802008701948BD
:109C500024214170A2210170C178C906C90EC170CA
:109C60000321017142718179C906FCD48179090708
:109C7000890F0229FAD14021417181790907890FA1
:109C80000229FAD181794906FCD51A21017081791E
:109C90000907890F0329FAD17047000000810440A9
:109CA000008004400000011040900440FFF8FFFED7
:109CB0000050064000400640BFF34F8F0349024862
:109CC000C860BFF34F8FFEE70400FA0500ED00E027
:109CD00038B5254D2C79E878800601D420208443BE
:109CE000E878000601D480208443200616D51F485A
:109CF00002F05DFD002800D00120E7221CA102F047
:109D0000B1FC1A4802F074FDE871184802F04FFDEA
:109D1000002803D1E8784006400EE870A00605D57B
:109D20006007800F03D0E8796946087038BDED7987
:109D30001B4802F02BFD0446132804D92946184875
:109D400002F092FD38BD02F045FE002807D0132C2A
:109D5000F8D1132213A1124802F0D7FD38BD1048E4
:109D600002F046FDEAE7000000B00640CC130020F8
:109D70002E2E5C2E2E5C2E2E5C736F757263655CCE
:109D80006869635F68616C5C667265657363616C6A
:109D9000655C6B6C32367A5C756172742E630000A0
:109DA000DC1500203C4441504C696E6B3A4F76659F
:109DB00072666C6F773E0A00F8B52E4E0024357837
:109DC0000095280741D5317C0A090807C00F4B07C9
:109DD000DB0F154605431AD1950040002818C0181E
:109DE000254BC0001D5CAD062D0F012D0FD1C518F0
:109DF0006F88002F0BD1214FBA5C6A801A5C520623
:109E000001D5882200E0C8221A5401200143EFF353
:109E10001080C507ED0F72B6194A184F143FB86885
:109E200011541521401CFEF71DFCB960002D00D116
:109E300062B608203070002C02D1307D800601D53A
:109E4000012400E000243578BBE700990B48294342
:109E5000083804F00AFC002C01D0012000E00020AA
:109E6000064914390A7810430870357002F056FB21
:109E7000F8BD000080200740001A002090F1FF1F6D
:109E8000A01F002000207047034801694069081A9C
:109E900002490988081A7047DCF1FF1F6623010098
:109EA00070B50B4D0C460346696B286B88420BD985
:109EB000401A844200DD044622461846FEF704FBA1
:109EC000686B0019686300E00024204670BD000044
:109ED000DCF1FF1F00207047F8B5184F0C4606460E
:109EE00079693869401A16490988081A002801DC7E
:109EF0000020F8BD844200DD0446FA69B8690025F7
:109F000090420DD30F4A031951188B4208D30D1AF2
:109F10002A463146FEF7D8FA76190A48641BB8611A
:109F2000002C06D022463146FEF7CEFAB869001959
:109F3000B8613969601909183961F8BDDCF1FF1F92
:109F400066230100EE18002010B5054C606800285B
:109F500005D10120606000F005F80020606010BDB0
:109F6000DCF1FF1FF8B5234CA06800283DD06169E3
:109F700020690026421AE06811460143002935D0C5
:109F800021461D4FC9691D4D002A10D0A06981428C
:109F900005D338888B182818834200D3421A1848F2
:109FA000007843001748C05A904200DA024616482B
:109FB000E66000788023184302F0D8FAE1690918B6
:109FC000E1616269121862613B88EB188B4200D133
:109FD000E561216991420BD1094909784A00094993
:109FE000895A814204D10120E060F8BDA660F8BD25
:109FF000E660F8BDDCF1FF1F66230100EE180020CB
:10A000001FF2FF1F6A2301006423010010B50C4CEE
:10A01000206A002803D0A06A401CA06210BD012065
:10A020002062606200F00EF8002060622062616BC6
:10A03000206B8842F2D0401AFFF74CFF10BD0000A1
:10A04000DCF1FF1F10B5134C1348216B154B0A1A96
:10A0500012480088821A124800784000185A82423A
:10A060000EDB1148007801F01BFE216B08182063FD
:10A07000A06A00280CD0616A002909D1401E06E0C0
:10A080000120E062606A002802D0A06A401CA06241
:10A0900010BD0000DCF1FF1F2E1900206823010015
:10A0A0001FF2FF1F6A2301006523010010B504465B
:10A0B000400702D52046FFF7A9FF200702D520461A
:10A0C000FFF742FF10BD00207047002070470000DE
:10A0D00010B50C4800F042F8002812D00948FEF7ED
:10A0E000A8FA0949020A08704A70020C8A70000E28
:10A0F000C870044802790A7142794A71807988717E
:10A10000012010BD14F2FF1FEC17002010B51048FD
:10A11000002444608460C46004610E49816144612C
:10A12000046244628462C462C1610B490163416399
:10A13000014604804B203831C001FEF78BFA0448F9
:10A140000821383004714471817100F019F810BD94
:10A15000DCF1FF1FEE1800202E19002070B5044618
:10A16000064D21462868FEF775FA2879A0716879AE
:10A170006071A8792071012070BD0000A0F2FF1F5E
:10A1800010B506F015FB03F0CBFE012010BD10B595
:10A1900006F050FB012010BD0120704710B50446A9
:10A1A000FEF747FA06490860A0790871607948719E
:10A1B000207988710020C871084606F051FB10BD57
:10A1C000A0F2FF1F10B51148002444608460C460F1
:10A1D00004610F4981614461046244628462C46223
:10A1E000C1610C49016341630480FFF7D0FF074957
:10A1F0004B203831C001FEF72DFA044808213830D1
:10A20000047144718171FFF7C9FF10BDDCF1FF1FBC
:10A21000EE1800202E19002010B5FFF7D3FF10BD57
:10A2200070B51B480078002831D01A4C0025206AF0
:10A23000012600280AD1616B206B884206D116499D
:10A24000884203D02163E56225626163A06A002829
:10A2500010D0206A00280DD1E06A00280AD12662B9
:10A26000FFF7F0FE2562616B206B884202D0401A36
:10A27000FFF730FEA1686068084308D16169206972
:10A28000884204D06660A660FFF76CFE656070BD12
:10A290001DF2FF1FDCF1FF1F2E190020B0B50D4C81
:10A2A0000D4F002806D0BC4600DF2060002006F0DD
:10A2B00073F80CE0BC4600DF2168401AFF212D3105
:10A2C000884201D3012000E0002003F037FE012086
:10A2D000B0BD00009CF2FF1FF1F3000000207047AA
:10A2E0000020704710B502490880FFF755FF10BDE8
:10A2F000DCF1FF1F10B50B48FEF79BF9094C00027B
:10A30000E178000A090608430749FEF7A3F9064861
:10A310002179017161794171A1798171FFF73EFF66
:10A3200010BD0000EC17002014F2FF1F01078A0E79
:10A33000044910B551180A78FD231A400A7002F03A
:10A3400087F810BDC020074010B501464A790B7947
:10A35000807811021943020601D4024A115402F016
:10A3600077F810BD90F1FF1F704710B500F016FB95
:10A3700010BD0000094A094980320028087D04D038
:10A38000012318430875102005E0400840000875B7
:10A39000107AEF21084010727047000080200740BB
:10A3A00010B50C4C0C48A2880078824200D90246B5
:10A3B000002A03D107490020143908718020216840
:10A3C00002F0D4F8216809182160A188081AA08039
:10A3D00010BD000030F2FF1F4423010010B5064CF1
:10A3E0000020A288216801F05BFC21680918216027
:10A3F000A188081AA08010BD30F2FF1F704700002E
:10A400000749020605D50007800E40180178FA2298
:10A4100003E0800040180178F62211400170704777
:10A42000C02007400749020605D50007800E4018E6
:10A430000178052203E080004018017809221143C9
:10A4400001707047C0200740F8B504466F4F704D4B
:10A45000704E800720D502F057F83878C009FFF712
:10A46000CDFFF888A88038784106890F04D00129EB
:10A470005CD0022975D169E079780B0002F0A2F86E
:10A480000C070D7113711928712D333B4A7101F0BE
:10A49000A9FD1FE0FFF784FF70E0002004E002F058
:10A4A00047F85D483DE0012001F0DEFD002858D06E
:10A4B000F5E7C006C00E54D1B8788021084330704B
:10A4C0004006400E012102F009F802F031F855E093
:10A4D00001F076FC002844D0DCE7C006C00E40D175
:10A4E0004C48401C14E001F013FE002839D002F063
:10A4F0001FF84A4815E0C006C00E012831D1707817
:10A5000000282ED03879B17888422AD244494018A0
:10A510002860BFE701F0C0FE002822D002F008F852
:10A5200040480068002829D0804727E0C006C00EB8
:10A5300017D0012815D100F017F900281ED100F01E
:10A540006FF900281AD100F0BBF808E0C006C00E71
:10A5500007D100F09FF9002810D100F0E7F900289A
:10A560000CD13878C00904D1F888002801D0002027
:10A5700000E0802001F0BCFF0020A880600704D527
:10A580003878C0090DD001F0DBFF200733D53878CB
:10A59000C00927D0A888317908432CD0FFF700FFE5
:10A5A00029E0A8880028F0D0FFF718FFA888002825
:10A5B000EBD138784106890F0ED001290CD1C006A5
:10A5C000C00E09D0012807D100F05CF80028DCD1CA
:10A5D00000F02AF80028D8D1802001F089FF00205F
:10A5E000A880D2E73078010605D54006400E3070CD
:10A5F000002101F073FF600602D50020FFF796FEF0
:10A60000200602D58020FFF791FEF8BD38F2FF1F2B
:10A6100030F2FF1F1CF2FF1FCC230100C4230100F6
:10A620006FF1FF1FC823010010B51349134A0879C1
:10A630001278904203D0124A1278904219D1487889
:10A64000002804D0022805D0202812D10EE0FFF700
:10A6500045FE05E0C878897800020843FFF740FE10
:10A66000002806D001F064FF012010BDFFF742FE74
:10A67000F6E7002010BD000038F2FF1F6223010042
:10A680006323010010B50B490B4A087912789042F8
:10A6900003D00A4A127890420AD14878092807D193
:10A6A00000F07EFB002803D001F042FF012010BD26
:10A6B000002010BD38F2FF1F452301004623010092
:10A6C00070B52449244A08791278904203D0234A6D
:10A6D000127890423BD11F484978C27883781002A3
:10A6E0001F4C204D1843042920D008DC00290FD02E
:10A6F00001290FD002290BD0032928D111E02029EC
:10A7000006D0212919D022291AD023291FD11AE0D5
:10A710002C6010E0FFF7D9FC05E02C60FFF740FE4D
:10A7200009E0FFF7D0FC0028F7D110E0FFF7AAFB03
:10A730000BE001F0FDFE012070BDFFF7C9FCF2E760
:10A74000FFF7D0FD01E0FFF7A9FD0028F1D10020BF
:10A7500070BD000038F2FF1F622301006323010077
:10A76000EC17002030F2FF1FF8B5254E254930794F
:10A770000978884203D02449097888423DD170780D
:10A78000224C234D234F030001F01CFF0C370723FD
:10A790002D37373737371826333700F01FFA0028A0
:10A7A0002BD0F078012802D0032803D003E01A4808
:10A7B000206000E02560FFF7F3FD12E0F07802284A
:10A7C00002D0032803D00CE01448206009E0256083
:10A7D00007E000F0EBF908E000F0BAFA0BE001F056
:10A7E000A7FE0120F8BD00F0EFF9002805D0276092
:10A7F000E1E700F0CBFA0028F1D10020F8BD00001D
:10A8000038F2FF1F452301004623010030F2FF1FED
:10A810007AF1FF1FEC1700202D1800206E18002081
:10A8200010B51848184A01791278914227D1427818
:10A830000146C8788B7800021843CB798C791902CD
:10A840002143FE2A0CD0FF2A19D1002817D1002954
:10A8500015D101F065F9002811D001F069FE0CE076
:10A8600000280CD101290AD100F04AFE002806D0A8
:10A87000074906480860FFF793FD012010BD00203E
:10A8800010BD000038F2FF1F58230100EC17002014
:10A8900030F2FF1F70B51F4D1F49687809780026F8
:10A8A000884235D1687929790002084302282FD1DE
:10A8B000AA781A4C002A2BD0002004E02178002925
:10A8C00000D00C19401C411C8A42F7D8207800287F
:10A8D00019D003F01DF90146E01CFDF7E9FD104A0F
:10A8E00001261460E979AB79207809021943814285
:10A8F0000BD90C4990800978491E084206D10A49B3
:10A900000120087002E0002602E09180FFF748FD78
:10A91000304670BD38F2FF1F6E23010030F1FF1F7B
:10A9200030F2FF1F4423010020F2FF1F10B5154A2B
:10A930001549507809780024884220D1507911793E
:10A940000002084307281AD1114B10481860417AB9
:10A95000007A09020143D079927900020124104360
:10A96000884209D90B4899800078401E014204D1E1
:10A9700009490120087000E09880FFF711FD20468A
:10A9800010BD000038F2FF1F6F2301000A240100F0
:10A9900030F2FF1F4423010020F2FF1F074800216F
:10A9A0004170C16001614161418081808161C1610B
:10A9B000C1800181016241817047000040F2FF1FA8
:10A9C000F8B5494EB0887188484F00257C1C8842F4
:10A9D00018D3B069002815D17561B5800123397885
:10A9E0007A1C184606F00CFA70807088002809D08E
:10A9F0003F4877610078012801D8746102E07088CF
:10AA0000401C7080708800283AD1F068002801D07E
:10AA1000F56035E03069002832D0354909780129E0
:10AA20000ED83D70B58002237A1C0021012006F06B
:10AA3000E7F970807088002800D0746135611FE0EC
:10AA40003C780127202C00D300243946A140014244
:10AA50001AD0601CC1B2254A02231170B5800120B2
:10AA6000521C06F0CDF970807088002804D01F4871
:10AA700070617088401C70803069A740B8433061B5
:10AA80007088002806D102E0641CE4B2DAE7B069FD
:10AA9000002826D07088B188164F401A84B23878C2
:10AAA00041001548405AA04200D204461348802174
:10AAB000007822460843716901F058FD7069104919
:10AAC00000197061B088001980B2B080098888428E
:10AAD00008D2387841000848405AA04202D10120EB
:10AAE000B061F8BDB561F8BD40F2FF1F2C18002021
:10AAF000522301001FF2FF1F4E23010047230100D4
:10AB000054230100F8B51B4C002720891A4D1B4E19
:10AB1000002802D1E5613188E180E1880A1A1848ED
:10AB2000E169007801F0BCF8E16980B20918E161DF
:10AB3000218909188BB22381002809D031888B42E2
:10AB400006D21049104A09784900515A814210D959
:10AB50000E48017801200129009003D80021064AFF
:10AB6000022003E029786A1C02205B1E06F0D0F95F
:10AB70002781F8BD40F2FF1F6D1800205623010009
:10AB8000482301001FF2FF1F4E2301005323010041
:10AB900010B50446000702D52046FFF711FF6007F5
:10ABA00002D52046FFF7AEFF10BD00000348044960
:10ABB0008078085C034908700120704738F2FF1F55
:10ABC00078F1FF1FEC17002010B506F017F90249C5
:10ABD0000870012010BD0000EC17002010B50B49D3
:10ABE0000022C878012804D0022804D0032806D106
:10ABF00003E0074A02E0002010BD064A521C897893
:10AC0000002306F0FDF8012010BD000038F2FF1F00
:10AC10002C18002079F1FF1FFEB544480078002869
:10AC20007ED0434E002031788446481C3070414825
:10AC3000042300784200821893405B1E01929942DF
:10AC400003DB0021317001218C463B4A002511882D
:10AC5000FF2901D2491C118041003848405A364929
:10AC600000900988884200D10125354900200978E3
:10AC70008E4648E000216246002A0DD0314A135C1E
:10AC8000FF2B01D25B1C13542F4B1B5C002B03D0FA
:10AC9000125C9A4200D301212B4A0223145C019AD0
:10ACA000934022469A40009B9A4203DA002C01D03E
:10ACB000012200E00022002D06D0002A04D001234A
:10ACC000376983403B433361204B1B5C9C420CD073
:10ACD0001C4C245C9C4206D30124376984403C43CD
:10ACE000346100243470184C2354002909D0002A00
:10ACF00004D101213269814011433161114A00219F
:10AD00001154401CC0B27045B4D3002D02D00A4982
:10AD1000002008803069002806D07088002800E0F4
:10AD200002E001D1FFF74CFEFEBD00001DF2FF1F47
:10AD300040F2FF1F1FF2FF1F74F1FF1F4A230100A3
:10AD40005223010076F1FF1F77F1FF1F78F1FF1FFB
:10AD50000A480A498078C978002802D0084A8154F4
:10AD600009E0094B0020074A1B7802E01154401CFF
:10AD7000C0B29842FAD301207047000038F2FF1F9A
:10AD800077F1FF1F78F1FF1F5223010010B5034830
:10AD9000807806F0BBF8012010BD000038F2FF1FDC
:10ADA00038B50D490022C878012804D0022804D003
:10ADB000032806D103E0002038BD084A00E0084A15
:10ADC000521C00230093CB798C791B022343897892
:10ADD00006F09EF8012038BD38F2FF1F6D180020E4
:10ADE00079F1FF1FF8B5EFF31080C007C00F72B6FE
:10ADF000564D0021EC68E9602A78009229700028FD
:10AE000000D162B6E00708D001F0DCFA06F052F992
:10AE10004F480068002800D08047E00606D501F0C2
:10AE20009BFB4C480068002800D08047A00606D550
:10AE300001F046FB48480068002800D080476007C2
:10AE400004D546480068002800D08047022C09D16C
:10AE500043480168002902D04248007A88474148A7
:10AE6000FF210172200767D53F4FEFF31080C20723
:10AE7000D20F72B6A9686868884257D1012156E09E
:10AE8000EFF31081CE07F60F72B638490C5C15212E
:10AE9000401CFDF7E7FB6960002E00D162B620463A
:10AEA0002207D30F21066207090FD20F002908D10C
:10AEB0005C00A418E4003C5D0026A406240F0D2CC1
:10AEC0000AD08C005B00E3189A18D600BA5D92068F
:10AED000120F012A13D01DE028690221884328613E
:10AEE000387E4006400E3876387C4006400E387476
:10AEF0001F486E7001680029B7D0022014E00029B5
:10AF000002D1C007C00F687019480159002901D04B
:10AF100004208847B85D8006000F0928A5D1144891
:10AF200001590029A1D0082088479EE70021002A66
:10AF300000D162B60029A3D00098002804D00949A6
:10AF4000087DDF2210400875F8BD00007CF1FF1F6E
:10AF50007023010074230100782301007C23010089
:10AF60008023010080200740001A0020A01F00203D
:10AF70008423010010B51C48402303701B4841681E
:10AF80000522120411434160416B1A0311434163CE
:10AF900000F036F81648017B802211430173017BD3
:10AFA0000906FCD41349124C090A803C2177114947
:10AFB0000A0C0F4960390A740E4A120E0A75FF21F5
:10AFC00021700D490968002900D004210B4A12683C
:10AFD000002A00D00222114319221143217103706B
:10AFE000017B1943017310BD90F1FF1F00800440E5
:10AFF00000210740001A00207C230100802301006B
:10B0000001200249000608607047000000E100E0EE
:10B0100070B500F019F900282AD0164802240470EF
:10B020004470154E03203463307014480546FDF714
:10B0300000FB022808D9114920461F39FDF70AFBF9
:10B0400029462046FDF706FB0D4880210078224660
:10B050000843084901F08AFA2846FDF7EAFA316BFD
:10B06000401A2946FDF7F6FA044901200839087309
:10B0700070BD0000AE18002064F2FF1FA720002062
:10B080005923010010B510490878022808D0032878
:10B090000FD0042810D0052801D10020087010BD61
:10B0A0000A48C07B282801D0A828F8D100F06CFA03
:10B0B00010BD00F077FD10BD0548802100780843E1
:10B0C00000F08AFDF5E7000064F2FF1F80200020F9
:10B0D0005923010010B51D4A117800290FD001290C
:10B0E00010D01B48052900781BD0072927D000F075
:10B0F00073FD18490220087300F054FD10BD00F0E4
:10B100000FF910BD13481F38C07B2A2803D02F2801
:10B1100004D0AA28F5D100F015FB10BD00F0A2FA6A
:10B1200010BD012181400C480068014201D001207E
:10B1300000E00020094A0AA101F094FA10BD0020A5
:10B140001070106B1F28DAD010BD000064F2FF1FD2
:10B150005A2301009F20002028F2FF1F4104000015
:10B160002E2E5C2E2E5C2E2E5C736F757263655CCA
:10B170007573625C6D73635C757362645F6D73633A
:10B180002E63000010B5144C6068E060002801D008
:10B19000012010BD1148FDF74CFA002814D00F48CB
:10B1A0000838007B000604D50D488021007808434C
:10B1B00008E00A481F30FDF73CFA216B884203D0B3
:10B1C0000848007800F008FD044901201731087391
:10B1D00000F0E8FC002010BD64F2FF1F8820002072
:10B1E000592301005A23010010B5124801798F201C
:10B1F0000140080605D50807000F0122120482400D
:10B2000001E001228A400C480478802004438C42EB
:10B210000ED10A48006810420AD00948FDF709FA21
:10B220000849884204D10D220549204601F09EF9C3
:10B2300010BD000038F2FF1F5923010028F2FF1F44
:10B240009F2000205553425370B50C48FDF7F1F98B
:10B250000A4C02251734002808D020461F38007BEE
:10B26000000608D40648007800F0B6FC257300F00C
:10B2700099FC002070BD012070BD000088200020D6
:10B280005A23010070B51148FDF7D3F9104C216B1A
:10B29000884202D82063032000E0042020700D487B
:10B2A00080210078226B08430B4901F05FF90748C1
:10B2B0001F300546FDF7BDF9216B401A2946FDF701
:10B2C000C9F9024900201731087370BD8820002099
:10B2D00064F2FF1F59230100AE18002010B5064884
:10B2E000064902880648007800F0DAFC0549086340
:10B2F000FFF7F0FE10BD000060230100AE18002033
:10B300005A23010064F2FF1F10B50446400702D51E
:10B310000020FFF7E3FF200701D5FFF7B3FE10BDC4
:10B32000F8B5704E316B1F2901D20A4600E01F228A
:10B3300000206D4D6D4B02E01C5C2C54401C904273
:10B34000FAD36B48802200780127104300901F2910
:10B3500070D16548FDF76DF9664988426AD1281DAC
:10B36000FDF767F9604C1F34211DFDF773F9204686
:10B370001738FDF75EF921460831FDF76BF9687B58
:10B38000002804D1A87B002801D0102801D92773F8
:10B3900074E0E87B2A283BD020DC1A2847D00EDC5A
:10B3A0000428F4D006DC00283BD00328EFD100F0BD
:10B3B00075FBF8BD1228EAD100F0AAF8F8BD2328E1
:10B3C0003CD006DC1B282FD01E28E0D100F0CCF8A2
:10B3D000F8BD252835D02828D9D13BE09E2836D085
:10B3E0000EDC5528D3D004DC2F2842D03528CED10E
:10B3F00003E05A281FD09128C9D100F01DFCF8BDE8
:10B40000A12821D0A3284ED0A82823D0AA28BED175
:10B4100000F084FA0028F2D0287B00063BD4377075
:10B42000F8BD00F013FCF8BD00F0ECFBF8BD00F037
:10B4300047FAF8BD3BE000F011FAFAE700F0F2FA43
:10B44000F7E700F0C9FAF4E7FFF7E2FDF1E700F0F3
:10B450007DFBEEE700F062FA0028EAD0287B0006C8
:10B4600004D50220307000F08FF8E2E7224800781F
:10B4700015E0287C800704D40020207300F092FBA4
:10B48000D7E700F04BFA0028D3D0287B000602D47F
:10B4900037703762CDE7164880210078084300F006
:10B4A0009BFB0220E9E7009800F096FB6FE7104C49
:10B4B000009800F091FB2078104C0107090F012043
:10B4C0000004884021680C4D08432060287800F073
:10B4D00083FB287887402068074306202760307068
:10B4E000A7E7000064F2FF1F80200020AE180020B4
:10B4F00059230100555342435A2301002CF2FF1FE8
:10B50000024900200870012070470000EC1700205D
:10B5100010B5FFF799FE00281FD0104B00201870BF
:10B520008021597002219970D97020241C715871A2
:10B530009871D8710A48016808200A78002A02D058
:10B540001A54491C00E01C54401CC0B22428F4D3F7
:10B55000044924200863FFF795FE10BDAE180020B3
:10B560002CF1FF1F64F2FF1F10B50548C07CC10716
:10B57000044800D00121017300F014FB10BD00004D
:10B58000802000209F200020F8B5314D314FA9695F
:10B59000686A002688420AD338788021002408434C
:10B5A00000F01AFB2C48067300F0FCFA08E02B4868
:10B5B000007841002A48445AE86A844200D304468D
:10B5C000FFF7E0FD002800D10024A86A00282DD054
:10B5D000002C0ED0A96AE8698022411838781043FF
:10B5E000224600F0C3FFA86A0019A862E86A001B9F
:10B5F000E86229696869AA6A4143914203D1AE624F
:10B60000696A08186862144808300746FDF711F89F
:10B61000001B3946FDF71EF8002C06D0E86A00280A
:10B6200003D1032028700C480673F8BD002CE0D02D
:10B630002969E86A4018401EFDF714F86969024656
:10B64000884200D90A46E969686A05F0F3FCC1E757
:10B6500064F2FF1F592301009F2000201FF2FF1FEB
:10B660005C230100F8B5334C0025A169606A88426B
:10B6700008D331482563007800F0AEFA2F480573EF
:10B6800000F090FAFFF77EFD002806D0206B00281E
:10B6900024D0A06A002802D010E025631EE02169B2
:10B6A000E06A4018401EFCF7DDFF616902468842EF
:10B6B00000D90A46E169606A05F0BCFC0020204917
:10B6C000A76A266B08E0E3693A189A5C0B5C9A4219
:10B6D00001D0256202E0401CB042F4D3266BA06A80
:10B6E0008119A162E06A871BE762226960694243AF
:10B6F0008A4203D1A562616A081860620F48083067
:10B700000546FCF796FF801B2946FCF7A3FF002E99
:10B710000CD0002F02D02078052807D1206A0028FD
:10B7200005D000200549087300F03CFAF8BD01205F
:10B73000F8E7000064F2FF1F5A2301009F20002059
:10B74000AE180020F8B5384D384FA969686A002650
:10B75000884207D336482E63007800F03DFA3E73E6
:10B7600000F020FAFFF70EFD002800D12E63296BB0
:10B77000A86A40182969884206D9FF2201322DA102
:10B78000002000F06FFFF8BD0020334905E0AB6AF0
:10B790000A5C1B18EC69401CE2542A6B9042F6D3F9
:10B7A000A86A8018A862E96A891AE962002A25D085
:10B7B000002914D1002812D029694018401EFCF736
:10B7C00051FF69690446884200D90C462246E9695E
:10B7D000686A05F047FCAE62686A00190DE06969A5
:10B7E0002B690A465943814208D1E969686A05F024
:10B7F00039FCAE626969686A401868620B480830B3
:10B800000090FCF716FF2C6B0099001BFCF722FF41
:10B81000002CB8D0E86A002802D028780528B2D1D8
:10B820003E7300F0BFF9F8BD64F2FF1F9F200020B7
:10B830005A2301002E2E5C2E2E5C2E2E5C736F750B
:10B840007263655C7573625C6D73635C757362646F
:10B850005F6D73632E630000AE18002070B5FFF7B4
:10B86000F3FC002824D0FFF78DFC002820D01148DD
:10B8700000210170062242700F4B81701A7A082451
:10B88000D201C270017141718171C1710B481C6399
:10B890000546FCF7CEFE082808D9084920461F397E
:10B8A000FCF7D8FE29462046FCF7D4FEFFF7EAFC59
:10B8B00070BD0000AE18002064F2FF1FA72000201A
:10B8C00070B5FFF7C1FC002820D0FFF75BFC002813
:10B8D0001CD00F480321017000210E4B41701A7AD1
:10B8E0000424D2018270C1700B481C630546FCF72A
:10B8F000A0FE042808D9084920461F39FCF7AAFEF3
:10B9000029462046FCF7A6FEFFF7BCFC70BD0000F0
:10B91000AE18002064F2FF1FA7200020F8B52A48C7
:10B92000FCF787FE284D00BA040A113D287D240249
:10B930000443264E00207462B062E87B2F280AD0B0
:10B9400004DC28280BD02A281CD104E0A82810D019
:10B95000AA2817D109E0FFF715FC002830D0E87DB0
:10B96000A97D0002084344BA0CE0FFF70BFC002855
:10B9700026D01548001DFCF75CFE00BA040A287E9C
:10B9800024020443306944430F48F4620938FCF749
:10B9900050FE0D4F01260E3700280DD0A04210D0CA
:10B9A000287B000604D50A4880210078084301E07E
:10B9B0000848007800F010F93E7300F0F3F800201A
:10B9C000F8BD0120F8BD00009120002064F2FF1FA7
:10B9D000592301005A23010010B5FFF735FC002858
:10B9E0001AD0FFF7CFFB002816D00C4A0C489169FB
:10B9F000491E0B0E03700B0C43700B0A8370C17051
:10BA000011690B0E03710B0C43710B0A8371C17129
:10BA100008201063FFF736FC10BD000064F2FF1F22
:10BA2000AE18002070B5FFF70FFC00282ED0FFF7EE
:10BA3000A9FB00282AD016480021017041708170AE
:10BA40000821144AC17091690C240B0E03710B0C70
:10BA500043710B0A8371C1710221017211690B0CD0
:10BA600043720B0A8372C1720B4814630546FCF7DC
:10BA7000E0FD0C2808D9084920461F39FCF7EAFDEB
:10BA800029462046FCF7E6FDFFF7FCFB70BD0000F1
:10BA9000AE18002064F2FF1FA720002070B5FFF74A
:10BAA000D3FB00282ED01B487021017000211A4BB7
:10BAB00041705A68DD681446AC4306D00624847091
:10BAC000282404734173DA600AE0002A1BD0134A69
:10BAD000127B002A1BD00522827020220273417340
:10BAE000C1700171417181710A22C271017241728A
:10BAF0008172C1728173C173017441741220186321
:10BB0000FFF7C0FB70BD022282703A22E6E7817027
:10BB10000173E4E7AE18002064F2FF1F9F200020AD
:10BB200010B50549002008600449FCF793FD04495D
:10BB300007200870012010BD2CF2FF1F9F2000205D
:10BB400064F2FF1F10B5FFF7EBFF10BD70B5FFF7F4
:10BB50007BFB00281DD00F4820220270002141707D
:10BB6000C1770D4C0320226320700C48802100789F
:10BB70000843084900F0FAFC09480546FCF759FD5E
:10BB8000216B401A2946FCF765FD0549012008395B
:10BB9000087370BDAE18002064F2FF1F5923010026
:10BBA000A720002010B508490848FCF753FD0848B5
:10BBB000802100780D220843034900F0D7FC054995
:10BBC0000520087010BD00009F20002055534253EF
:10BBD0005923010064F2FF1F10B5044600F088FCF1
:10BBE000200605D52107090F01200004884001E047
:10BBF0000120A04002490A681043086010BD0000FF
:10BC000028F2FF1F10B50A48817C04461F34002922
:10BC100004D001202073FFF7C5FF10BDC07C05498B
:10BC2000C007C00F486005F01BFA0020F2E70000D3
:10BC30008020002064F2FF1F10B503490020087324
:10BC4000FFF7B0FF10BD00009F20002010B5104886
:10BC5000FCF7EFFC0E4C173400280FD020461F389D
:10BC6000007B000604D50B4880210078084301E0E2
:10BC700009480078FFF7B0FF012004E0FFF782FADF
:10BC8000002803D000202073FFF78CFF10BD0000B8
:10BC900088200020592301005A230100704700002A
:10BCA000F7B5074682B0002000903807860E33486B
:10BCB000F500281801904488002F15D130484078AD
:10BCC000002809D07008012181402D48103002F071
:10BCD000D8FC002005B0F0BD2848405D8006000F6C
:10BCE0000D2801D1012000900498A04206D2FF2225
:10BCF000EF3224A1002000F0B5FC049C1F4A002074
:10BD0000B101A032891803E0039A0B5C1354401C64
:10BD1000A042F9D31A481430C15D0198174F4180F1
:10BD2000174876080069795DF040C0074906C00FE2
:10BD3000C90F88420FD10398C1798279080200990E
:10BD40001043002901D000280CD001210C48B1403B
:10BD5000103002F096FC0A480069F040C00708D095
:10BD6000C82007E006480121C943103002F071FCE9
:10BD7000F1E7882078552046ACE70000001A002043
:10BD80007CF1FF1F2E2E5C2E2E5C2E2E5C736F75A9
:10BD90007263655C6869635F68616C5C6672656547
:10BDA0007363616C655C757362645F6B696E657407
:10BDB00069732E630000000010B5FFF715FA10BD7F
:10BDC0007CB5534B534D1878534CC006C00E02D06F
:10BDD000012875D185E05149D8780E784D49CA7847
:10BDE0001C318978062810D006DC012809D00228E9
:10BDF00015D0032864D149E007282FD00F285FD140
:10BE00005FE047482060122069E0002E7ED0002AC3
:10BE100003D0444820600A2061E04348FAE7002E3E
:10BE200001D1012A72D0002A03D04048009000209E
:10BE30000CE03F48FAE7009A1378002B05D0D3783E
:10BE400096781B0233439A180092401C8142F2D12B
:10BE500000980178002959D020603CE0002E55D090
:10BE6000002A03D03348009000200CE03248FAE763
:10BE7000009A1378002B05D0D37896781B023343B1
:10BE80009A180092401C8142F2D1E1E72B480090C1
:10BE9000032901D0002009E001F094FE0DE0009993
:10BEA0000A78002A01D051180091401C99788142EB
:10BEB000F5D100980178002928D0206000780EE0A4
:10BEC00024E01F48007800281FD01E480090206002
:10BED000017800291AD0C1788278080210430190B5
:10BEE00005E001A9684600F031F800280DD0A188CE
:10BEF0000198814208D980B21349A0800978491E6F
:10BF0000084201D10120287101207CBD00207CBDA8
:10BF100038F2FF1F1CF2FF1F30F2FF1F3F2301000A
:10BF2000F6230100092401000824010079250100FD
:10BF3000ED2401007B2501007A2501007C2501000C
:10BF400040230100B42401004423010070B51A4AC3
:10BF50001A4CD3781A4A25781478174A194E127950
:10BF6000212B02D0222B24D118E0AA4201D0A242D8
:10BF70001FD1154A1378154A002B127801D1012AD6
:10BF800017D0002A08D0124A02601046114A1288BF
:10BF900080183060092009E00F4AF5E7AA4201D075
:10BFA000A24206D10D4830600D480088086001208B
:10BFB00070BD002070BD000038F2FF1F4523010056
:10BFC0004623010030F2FF1F3F2301001FF2FF1F35
:10BFD00079250100F4230100ED240100D0230100A4
:10BFE000F223010070B51D481D4B0078C106C90E33
:10BFF0000AD01D461948143D1A4C6A780079012967
:10C0000006D0022928D10AE015480E38186021E030
:10C01000002A21D0A97888421ED2002016E08F2164
:10C020000840010605D50607360F01210904B14075
:10C0300001E001218140002A01D100070CD1A8684C
:10C04000084209D0E868084000D001202070000AAA
:10C0500060701C60012070BD002070BD38F2FF1FB1
:10C0600030F2FF1FEC17002070B5274B02461878FE
:10C070001946C0064988254EC00E04D001282BD091
:10C08000022829D111E0012926D10224002A05D055
:10C09000012000F069FAF088204304E0002000F05D
:10C0A00063FAF088A043F0802CE01C798F200440D4
:10C0B000200605D52007000F01252D04854001E04D
:10C0C0000125A5407078002806D0200704D0B0686C
:10C0D000284201D0002901D0002070BD002A05D0DF
:10C0E000204600F005FAF06828430AE0306928424B
:10C0F00008D12046FEF71AF92046FFF75DFEF068EA
:10C10000A843F060012070BD38F2FF1F1CF2FF1F32
:10C11000F8B55A4800260178C906C90E7ED1574F96
:10C1200080781C3F00287FD0554801783846C07879
:10C13000002901D1012871D0002801D0514C6CE0B8
:10C14000514C6AE06078022804D0042846D00528C3
:10C1500061D145E0494861798078814239D1787070
:10C160002079B8704A490020484A0B8802E0002133
:10C170001154401C9842FAD301250120B968A84007
:10C18000084202D02846FEF73BF901200004B968B6
:10C19000A840084204D0284680210843FEF730F921
:10C1A0006D1C102DE9D33B48B8600020F860386161
:10C1B0003D460120FEF7D8F8E079400604D5E9882D
:10C1C00001200143E98026E0E88840084000E8803B
:10C1D00021E0E078A178000208431DE0E6781AE04B
:10C1E000002E18D1A5788F200540280605D52907EF
:10C1F000090F01200004884001E00120A840B9682F
:10C2000001432046B960FEF79FF82846FEF70AF979
:10C21000284600F01DF92078041901E029E003E028
:10C22000207800288ED11FE0002501247D70802613
:10C230000120B968A040084202D02046FEF7E0F88D
:10C2400001200004B968A040084203D020463043D2
:10C25000FEF7D6F8641C102CEAD3FD600D483D6152
:10C26000B8600020FEF780F804487978807888422A
:10C2700001D00020F8BD0120F8BD000038F2FF1FFA
:10C280003F23010079250100ED2401006FF1FF1F1C
:10C290004223010001000100F0B585B000274448A9
:10C2A0000397019700783E46C006C00E01287DD155
:10C2B0003F491C394878002875D0002002903D483D
:10C2C00002780846C078002A01D101286ED00028E3
:10C2D00001D0394C63E0394C61E06078022804D029
:10C2E00004280DD0052858D11CE0314861791C384C
:10C2F0004078814251D0E078A178000208434DE0B7
:10C30000A778E6780020019029480179B94244D104
:10C310008078B04241D1012002902948C15D03914B
:10C32000C6553AE022490879B84236D1A0788F2222
:10C33000104000900006009804D50007000F01256A
:10C340002D0400E0012585408878B04214D11848BA
:10C350001C38816829438160C168A943C1602046B7
:10C36000FDF7F2FF0098FEF75DF8009800F070F816
:10C3700001982843019010E0039886420DD101985E
:10C3800028420AD10A481C388168A9438160C168E3
:10C39000A943C1600098FEF733F82078041920788B
:10C3A00000289AD1029805B0F0BDFFE70020FAE717
:10C3B00038F2FF1F3F23010079250100ED24010021
:10C3C0006FF1FF1F70B501261A483606066001207E
:10C3D000194D0024810049190C70401C1028F9D314
:10C3E00015211648FCF723F9154816494460846066
:10C3F000C4600470447040224A800A46A0324A60F9
:10C40000C8220A700C72104ACC614A610D21297051
:10C410000E49016108484038017D0222114301752F
:10C42000FF210170017201730476024880380660B2
:10C4300070BD000080E100E0C0200740A01F002088
:10C440007CF1FF1F001A0020201B00205555555578
:10C45000F8B50546154F2C073E4600060121A03EC3
:10C46000240F00280EDA6000401C8140104802F0C2
:10C47000FCF82002C119600180198031416100215E
:10C48000C161F8BD68008140C943094802F0E1F884
:10C4900007486101001D425D881942802202D219BD
:10C4A00042608822725400210172F8BDA01A002057
:10C4B0008CF1FF1F10B5FDF7AFFEFFF743FB10BD7A
:10C4C00002480179DF221140017170478020074046
:10C4D00010B5FEF7A1FBFDF7A3FE10BD002903D1A7
:10C4E00040060249400E0876704700008020074051
:10C4F0000007810E034808180178022211430170D9
:10C5000070470000C020074010B5082202490020F3
:10C51000FFF7C6FB10BD000038F2FF1F10B503483F
:10C5200081680120400201F0B7FC10BD60F0FF1FE0
:10C5300010B500221146802000F018F810BD000050
:10C5400010B50348034902780020FFF7A9FB10BD8E
:10C5500044230100EC1700200248017920221143F6
:10C56000017170478020074070470000F8B5000750
:10C57000114F840E1646A41CE200D01946803D4699
:10C580000023A001A035451902E0C85CE8545B1CFB
:10C59000B342FAD3094960080969C140C90701D00B
:10C5A000882100E0C821B95401218140034810309E
:10C5B00002F067F83046F8BD001A00207CF1FF1F3A
:10C5C0000020704730B47446641E2578641CAB426A
:10C5D00000D21D46635D5B00E31830BC184710B500
:10C5E000002A06DA52005208D21DD308DB001022BE
:10C5F00003E0D21C93089B000C22002B02D09C1855
:10C600008C4201D9012010BD82188360411802605C
:10C610004160C91AD018884202D810600246F9E772
:10C620000020106010BD0000B0B5044602F044FFC9
:10C63000002804D0034F0249BC46206800DFB0BD8B
:10C64000FFFF0000A5EF0000B0B5044602F034FF84
:10C65000002803D0024F2068BC4600DFB0BD0000B8
:10C66000FDEE0000F8B516460F4600281BD1EFF38B
:10C670001080C507ED0F72B600231A4619461846FA
:10C6800000F006FA040003D13146384600F044FABF
:10C69000002D00D162B6002C05D1EFF30380C00657
:10C6A00001D104F0D1FFF8BD7047000010B5282279
:10C6B0000D490E48FBF70CFE05F09CF80C4805F000
:10C6C00093F804F095FE0B49012208600A495202D2
:10C6D0000A600A4A012111600949400A08600A49B2
:10C6E0000848086010BD0000641F0100D405002048
:10C6F00059D0000098F2FF1F74F2FF1F78F2FF1F5D
:10C700007CF2FF1FD403002080F2FF1F00B591B020
:10C71000FDF7BAFB402801D9402001E000280DD0E8
:10C7200081B2684604F07CF8010007D06846FDF746
:10C73000D3FB002802D0012001F0DAFB04F0FEF860
:10C740000146402801D9402101E000290DD068466A
:10C75000FDF7A6FB002808D081B2684604F0CEF8A9
:10C76000002802D0012001F0C3FB01F0D9FB11B079
:10C7700000BD0000044841788078814201D001204A
:10C780007047002070470000F4F0FF1F30B50546E9
:10C79000EFF31080C407E40F72B6284600F007F8E4
:10C7A000A968081A401E002C00D162B630BDEFF314
:10C7B0001081CB07DB0F72B606C808388A4201D356
:10C7C000501A02E080681018401A002B00D162B69F
:10C7D0007047EFF31083DB07DB0F72B68260C16036
:10C7E000002101604160002B00D162B6704700005B
:10C7F00070B50446EFF31080C507ED0F72B603CC99
:10C80000083C884201D0012000E0002043220DA115
:10C81000FFF728FFE16820680E5C401C2060A168DB
:10C8200088420AD3884201D1012000E0002048223A
:10C8300004A1FFF717FF00202060002D00D162B691
:10C84000304670BD2E2E5C2E2E5C2E2E5C736F75C6
:10C850007263655C6461706C696E6B5C6369726362
:10C860005F6275662E63000070B50446EFF31080BA
:10C87000C507ED0F72B66268E06881546068401CBD
:10C880006060A16888420AD3884201D1012000E09B
:10C890000020312209A1FFF7E5FE0020606003CCF3
:10C8A000884201D0012000E00020362203A1FFF7DA
:10C8B000D9FE002D00D162B670BD00002E2E5C2E78
:10C8C0002E5C2E2E5C736F757263655C6461706C98
:10C8D000696E6B5C636972635F6275662E630000EC
:10C8E000F8B514460E460746FFF761FF844200D2B2
:10C8F00020460546002404E03846FFF779FF30550E
:10C90000641CAC42F8D32846F8BDF8B514460E4670
:10C910000746FFF73BFF844200D22046054600242D
:10C9200004E0315D3846FFF79FFF641CAC42F8D34A
:10C930002846F8BD10B50C48C0780121C009484010
:10C940002A220AA1FFF78EFE144901246402084638
:10C9500022461038FFF73DFF11492246084610389D
:10C96000FFF737FF10BD000000B006402E2E5C2EF2
:10C970002E5C2E2E5C736F757263655C6869635FF5
:10C9800068616C5C667265657363616C655C6B6C39
:10C9900032367A5C756172742E630000DC130020FD
:10C9A000EC15002010B500F089FC10BD10B500F0AA
:10C9B00085FC10BD02488079002800D00120704716
:10C9C000642000200248C079002800D00120704770
:10C9D000642000200248007A002800D0012070471F
:10C9E00064200020F8B54B211F48FBF71EFE4B27A3
:10C9F0001E48FBF71EFE1C4C1D4E1C4D4034B04221
:10CA000013D168792A79010211434B2901D20A46D0
:10CA100000E04B224B2901D90F4600E04B27134978
:10CA20001148FBF751FD0020E0714B210F48FBF747
:10CA3000FCFD0E493046FBF70DFE2F71390A697176
:10CA400009494122C91DE81DFBF73EFD607A227AA3
:10CA500001020648114340300172090A4172A17A6D
:10CA6000817200F08BF8F8BD18200020002F002004
:10CA7000646C766B10B541210448FBF7D6FD034882
:10CA8000002139300172417210BD0000072F0020D3
:10CA9000FFB581B01D4616460F461A48FBF78CFCC1
:10CAA000441C0198002802D03946FBF7BEFD002047
:10CAB000002E00D03080002D00D028701149C91FF1
:10CAC000C87900281BD0BC4201D8224602E0E01BF6
:10CAD00041183A460B4C0198C91D3934002804D03E
:10CAE000607A237A000218433080002E02D0019829
:10CAF000FBF7EAFC002D01D0A07A2870012005B0D8
:10CB0000F0BD0000072F002002488079002800D0E7
:10CB100001207047002F0020F3B581B00746FBF7D6
:10CB20004BFC124D441C41263146E81DFBF77DFDB0
:10CB3000412C02D83946224602E0413CE1193246F6
:10CB4000E81DFBF7C1FC094C029840342072000A32
:10CB5000607200F00EF9002801D0012004E000F01E
:10CB60000AF9002800D00220A072FEBD002F00208C
:10CB70000149887170470000002F002070B5002225
:10CB800011461046FCF758FD092220492048FBF7C2
:10CB90009BFC204C22781046627812021043A27847
:10CBA000E1781204104309061B4D0843A8420FD137
:10CBB0006079217900020843092804D2607921793B
:10CBC00002020A4300E0092212491148FBF77CFCEB
:10CBD0000F492846FBF73EFD0D4909208880207843
:10CBE0000146607800020143A07800040143E07828
:10CBF00000060143A94205D160792179000208436A
:10CC0000092802D2024801F04BFC70BD5E260100EB
:10CC10006420002000FC0100646C766B10B50349B1
:10CC20008871084601F03CFC10BD00006420002023
:10CC300010B50349C871084601F032FC10BD000070
:10CC40006420002010B503490872084601F028FC52
:10CC500010BD000064200020F8B50024E4430F4616
:10CC60000646002512E0705D082101F021FF000654
:10CC700044400A490820002C02DA64004C4000E0DD
:10CC80006400401E0006000EF5D16D1CBD42EADBBB
:10CC90002021204601F00CFFC043F8BDB71DC104A0
:10CCA000F8B50E4617462021C04301F001FF0446A7
:10CCB000002512E0705D082101F0FAFE00064440F4
:10CCC0000A490820002C02DA64004C4000E06400AD
:10CCD000401E0006000EF5D16D1CBD42EADB20218E
:10CCE000204601F0E5FEC043F8BD0000B71DC104B9
:10CCF00070B514460D460646FF2A07D8FF22DD32DE
:10CD00000AA10020FFF7AEFC022070BD00F0C6FCB7
:10CD1000002801D00E2070BD2A462146304600F082
:10CD20002DFE0028F7D01C2070BD00002E2E5C2E9A
:10CD30002E5C2E2E5C736F757263655C6461706C23
:10CD4000696E6B5C647261672D6E2D64726F705CCE
:10CD50006961705F666C6173685F696E74662E638B
:10CD600000000000C1060007000F002900DB0930A9
:10CD70007047002070470120704710B500231A4605
:10CD800000F0D6FA002800D0012010BD10B504F044
:10CD90003FFA012800D0002010BD0000F8B5164E63
:10CDA0001F2530780024AD02012806D0FF2237323B
:10CDB00012A10020FFF756FC0AE0B07802270028F5
:10CDC00008D0FF223D320DA10020FFF74BFC377049
:10CDD0000220F8BD204600F02DF8002802D0377060
:10CDE0001E20F8BD012080022418AC42F2D301209D
:10CDF000B0700020F8BD0000D0F0FF1F2E2E5C2E7A
:10CE00002E5C2E2E5C736F757263655C6461706C52
:10CE1000696E6B5C647261672D6E2D64726F705CFD
:10CE20006961705F666C6173685F696E74662E63BA
:10CE300000000000F8B5254E05463078012805D0E1
:10CE4000FE2223A10020FFF70DFC1AE00127BF02FC
:10CE500039462846FBF706FC0224002902D0FF22AF
:10CE6000073209E0F07800280DD0F168B06840186A
:10CE7000A84208D0FF220E3215A10020FFF7F2FBD6
:10CE800034700220F8BD01227F20D20380020121EC
:10CE9000954203D3854201D2002000E008460028D5
:10CEA00010D0F170F7602846B56000F0B3FF22287B
:10CEB00003D00028E6D03470F8BD284600F0EEFB21
:10CEC0000028F9D034701D20F8BD0000D0F0FF1FFD
:10CED0002E2E5C2E2E5C2E2E5C736F757263655C3D
:10CEE0006461706C696E6B5C647261672D6E2D6439
:10CEF000726F705C6961705F666C6173685F696EA8
:10CF000074662E630000000001208002704700005C
:10CF100010B5242804D2064980000858002805D1FD
:10CF2000E12204A10020FFF79DFB0AA010BD000034
:10CF30005C1E01002E2E5C2E2E5C2E2E5C736F75F7
:10CF40007263655C6461706C696E6B5C6572726F54
:10CF5000722E63000000000001460120242901D246
:10CF60000148405C704700001CF0FF1FF3B581B022
:10CF70000446009000E0641C2078402802D000287D
:10CF8000F9D15EE06078622848D012DC522854D093
:10CF900008DC422842D0442849D0482841D04D28B6
:10CFA00017D134E054283FD0552833D0562810D11B
:10CFB00040E0722841D006DC642838D0682830D0A0
:10CFC0006D2806D123E074282ED0752822D076282B
:10CFD00030D01DA52046FBF7EFF907462846FBF7A2
:10CFE000EBF90646A019029B009AC119D218891EB6
:10CFF000914225D2BA1EA11CFBF7CAFA3246294635
:10D000002046FBF761FA20780028B5D119E000F03E
:10D01000CDFD01E000F0D2FD0546DBE700F078FD34
:10D02000FAE700F0A3FDF7E700F0C4FDF4E700F035
:10D0300099FDF1E700F0CAFDEEE705480568C9E78C
:10D04000E4190098201AFEBD4552524F52000000CC
:10D05000401E010070470000F8B51E4615460C46FC
:10D06000074604F05DFC2048007803280CD01E48D9
:10D070002038022C09D0002C19D0012C04D10068D2
:10D08000A84201D103F0BAF9F8BD0068A842FBD16B
:10D09000304604F085F90446304604F087F9064628
:10D0A000384602F0D9FB03462246314617E038469F
:10D0B00002F0D2FB0328E7D0304604F06FF9800776
:10D0C000E2D4384602F0C8FB0746304604F068F95F
:10D0D0000446304604F06AF901463B46224628469B
:10D0E00003F062FAF8BD0000F4050020F7B51C4E0D
:10D0F0000446B0785502174600280BD129460198FE
:10D1000002F066FB032802D0214603F0F9F9B0785B
:10D11000002812D0124920394868A0420DD8C868AA
:10D12000A0420BD0A04208D90869401C00D10C6174
:10D130000869A04200D204460C61FEBDC8692A46B7
:10D140008018C861E019C860F078002803D000207A
:10D1500003F078FAFEBD2046019903F07BF9FEBD8D
:10D16000F4050020F0B585B018A109680491037892
:10D17000002104AA545C9C4226D0491C0329F9D3FF
:10D1800013A10A688E6896464A68CD6800239446C3
:10D19000C25C714664466F46039552C711466139B9
:10D1A000192911D9202A01D2052A0DD100216C4656
:10D1B000675C974208D0491C1029F9D35B1C0B2BE4
:10D1C000E6D3012005B0F0BD0020FBE7E50020001C
:10D1D000222A2B2C2E2F3A3B3C3D3E3F5B5C5D7C54
:10D1E00070B50446204600F01AF80546002D00D020
:10D1F00070BD044902480968884700BFF8E700008D
:10D200000C3000F024F1FF1F01680122920211434B
:10D210000160BFF36F8FBFF34F8F704770470028D7
:10D2200007D0C069002802D00068022803D06D2012
:10D230007047042070470020704710B5002806D0C2
:10D240005B1E194201D11A4203D0652010BD042093
:10D2500010BD03688B4204D84068891818188842AA
:10D2600001D2662010BD002010BD00000349884295
:10D2700001D06B2070470020704700006B66656B23
:10D2800010B50C4C70212170FFF7C9FF002807D1A1
:10D2900009492046096888472078810601D567201A
:10D2A00010BDC10601D5682010BDC007FCD06920A3
:10D2B00010BD00000000024020F1FF1F70B50E4DB0
:10D2C00000202C78002C0FD000212970A97800298B
:10D2D00001D000F001FB022C05D06978032902D0AF
:10D2E000002800D1212070BDFF22343203A100208C
:10D2F000FFF7B8F9022070BDA4F0FF1F2E2E5C2EA0
:10D300002E5C2E2E5C736F757263655C6461706C4D
:10D31000696E6B5C647261672D6E2D64726F705CF8
:10D32000666C6173685F6465636F6465722E630029
:10D330003EB51D460446302901D3012000E00020FF
:10D34000402212A1FFF78EF921460C2220316846B7
:10D35000FBF7BAF81A49019888420BD1194900988D
:10D36000884201D102203EBD1649FC3988420AD1CB
:10D3700001203EBD204603F025FF002801D1002DED
:10D3800001D003203EBD00203EBD00002E2E5C2EAD
:10D390002E5C2E2E5C736F757263655C6461706CBD
:10D3A000696E6B5C647261672D6E2D64726F705C68
:10D3B000666C6173685F6465636F6465722E630099
:10D3C000019996978F9E939BFFB581B007460024E5
:10D3D00004982546002813D00A98002810D00499F4
:10D3E000002008600A9906460860FFF7C2FC002882
:10D3F00012D00120C003022F04D0032F0AD013E063
:10D40000652237E00399002904D00299814201D0B6
:10D4100018240AE0064615E0FFF7ADFC002803D00B
:10D42000012F07D0032F0FD01924FFF7CBFA0028C4
:10D430000FD010E00398002804D00298002801D0F3
:10D440001724F2E70E4802E00E4886680E48056889
:10D45000EBE7012F04D0002C04D0204605B0F0BD2E
:10D460001924FAE7002D04D0049806600A98056094
:10D47000F3E79D2205A10020FFF7F4F80220EDE775
:10D48000601F0100B4F1FF1F2C1F01002E2E5C2E27
:10D490002E5C2E2E5C736F757263655C6461706CBC
:10D4A000696E6B5C647261672D6E2D64726F705C67
:10D4B000666C6173685F6465636F6465722E630098
:10D4C00010B50D4C2078002806D0AC220BA100200E
:10D4D000FFF7C8F8022010BDFF2230211448FBF7E7
:10D4E0007FF801202070002060706060A060E06024
:10D4F000A070E07010BD0000A4F0FF1F2E2E5C2E67
:10D500002E5C2E2E5C736F757263655C6461706C4B
:10D51000696E6B5C647261672D6E2D64726F705CF6
:10D52000666C6173685F6465636F6465722E630027
:10D5300058FBFF1FF7B5494F0546387884B01446AD
:10D54000012807D0C12246A10020FFF78BF8022056
:10D5500007B0F0BDF878002803D1BD600120FD6060
:10D56000F870B878002856D1F9688D4201D10120B1
:10D5700000E000200919F96000282FD078683021D8
:10D580000E1AA64200D91646424932460818059995
:10D59000FAF79AFF7868A41B801978600599AD198D
:10D5A00089190591302829D316D00020E3222CA117
:10D5B000FFF758F801233748BA687968FFF7B8FED3
:10D5C000787001A8009002AB01227878B968FFF763
:10D5D000FBFE002826D103E00120E7E70320EFE768
:10D5E000B87801267040FC221DA1FFF73BF8019896
:10D5F00000F00CF9002815D1BE7002E0B8780028C0
:10D6000013D024497A68B86800F070F8002809D16E
:10D61000B878002809D022462846059900F066F817
:10D62000002802D00321397092E77878012804D0CD
:10D63000022805D003280FD105E01F20800204E056
:10D640007F20800201E01448C0682919814203D379
:10D650000220387010207BE7002079E7A4F0FF1F3C
:10D660002E2E5C2E2E5C2E2E5C736F757263655CA5
:10D670006461706C696E6B5C647261672D6E2D64A1
:10D68000726F705C666C6173685F6465636F64651C
:10D69000722E630058FBFF1FB4F1FF1F10B5EFF3AC
:10D6A0001081CC07E40F72B6FBF70CFE002C00D102
:10D6B00062B610BD70B50E460500144613D0202189
:10D6C0001046FAF7B4FF2660E8686060A9686868E9
:10D6D000FAF7C8FFA0600420E06020616061A061EB
:10D6E000E061002070BD042070BD0000F7B5384F28
:10D6F0000446787800251646012805D07B2235A1FE
:10D700000020FEF7AFFF09E07869844208D2832247
:10D7100030A10020FEF7A6FF022078700220FEBD97
:10D72000F878002809D1204601F04AFF050002D010
:10D73000022078704AE00120F870254FBA687868B6
:10D740008118A14219D8B97800290BD1B9698B6821
:10D750002D499847050003D01D490220487035E047
:10D760000120B870FF222848B968FAF739FF20462F
:10D77000B968FAF777FF601A7860002E24D039690B
:10D78000F8684018A04204D8204601F019FF0500AF
:10D79000E2D10F4948688968201A0F1ABE4200D2A8
:10D7A000374619493A4608180199FAF78DFE002FB5
:10D7B00008D000200649E41988700198C019F61BAA
:10D7C0000190BAE70120F5E7014844612846FEBD13
:10D7D000B4F0FF1F2E2E5C2E2E5C2E2E5C736F7508
:10D7E0007263655C6461706C696E6B5C64726167C6
:10D7F0002D6E2D64726F705C666C6173685F6D6115
:10D800006E616765722E630088FBFF1F70B5234D44
:10D8100004466878002801D047222CE0002C29D04B
:10D820006068002826D0A068002823D0E06800287F
:10D8300020D0206900281DD0606900281AD0A06976
:10D84000002817D00121FF2289021548FAF7C8FEE7
:10D850000126AE700020E8706860A860E86028616A
:10D86000AC61686120688047040009D128780028ED
:10D8700007D010E04D220BA10020FEF7F3FE02209E
:10D8800070BDA86900698047040004D0A869406899
:10D890008047204670BD6E70FBE70000B4F0FF1FAC
:10D8A00088FBFF1F2E2E5C2E2E5C2E2E5C736F7558
:10D8B0007263655C6461706C696E6B5C64726167F5
:10D8C0002D6E2D64726F705C666C6173685F6D6144
:10D8D0006E616765722E630070B5194C0025607823
:10D8E000002802D0012807D010E0CE2215A1002088
:10D8F000FEF7B8FE022070BDA078002806D1A0690E
:10D900001D498368A268606898470546A069406819
:10D91000804706460121FF2289021748FAF760FE78
:10D9200001200021A070E1706160A160E1602161CF
:10D9300061616170002E01D0304670BD284670BD17
:10D94000B4F0FF1F2E2E5C2E2E5C2E2E5C736F7596
:10D950007263655C6461706C696E6B5C6472616754
:10D960002D6E2D64726F705C666C6173685F6D61A3
:10D970006E616765722E630088FBFF1F10B5EFF3C1
:10D980001083DC07E40F72B6FBF792FE002C00D187
:10D9900062B610BD8021017001780906FCD5704780
:10D9A000704700000346012201490020184700008B
:10D9B00008060020024800698007C017401C704715
:10D9C00040F00F400020704708B51A48816B1F22B5
:10D9D000520211438163184980150861086108618A
:10D9E000164A50608860002000F03AF8002000F0ED
:10D9F0002DF8002000F03EF8114801680423194377
:10DA00000160426910210A43426142690A4342614E
:10DA100042690A43426141691943416108488038BB
:10DA2000416902229143416106480090401E0090E6
:10DA3000FCD108BD0080044000C0044000A00440A8
:10DA4000C0F00F4040420F00704700001022034911
:10DA5000012801D04A6070478A607047C0F00F40CB
:10DA600010220349012801D04A6070478A6070473C
:10DA7000C0F00F4010220349012801D04A607047CE
:10DA80008A607047C0F00F4010B50C4CA0680028A9
:10DA900012D0401EA060206909498001411840222F
:10DAA000002003F0D9F920690521401CFAF7DAFDBE
:10DAB00021616068401C606010BD000008F0FF1F1D
:10DAC000C0F2FF1F70B50F4C00206060A060E060E6
:10DAD0000D492061FFF7C0F8606001200B49C003C9
:10DAE000FFF7BAF80125A060AD021F202946800289
:10DAF000FFF7B2F8E0607F2029468002FFF7ACF81C
:10DB0000206170BD40F0FF1FFC7B0000FC7B01002A
:10DB10000048704754F0FF1F0021064B0A6A01209D
:10DB20009A4200D00020496A034A914200D0002066
:10DB300070470000939D939B0199969700B5FFF75E
:10DB4000EBFF002801D00020806A00BD014840683A
:10DB50007047000040F0FF1F0148806870470000D8
:10DB600040F0FF1F00487047A0F4FF1F00487047B7
:10DB70005EF4FF1F0120C103054B0A6A9A4200D0E0
:10DB80000020496A034A914200D0002070470000FB
:10DB90008F9E939B0199969700B5FFF7EBFF0028A6
:10DBA00002D00120C003806A00BD00000048704719
:10DBB00051F4FF1F004870477FF4FF1F0048704773
:10DBC00020F4FF1F00487047A9F4FF1F004870476A
:10DBD00059F0FF1F70B5FFF775FF1F4800F0E8FE12
:10DBE00001F096FC1C4831212030FAF720FD1A483C
:10DBF0001A492030FAF75CFC174819A12030FAF7CF
:10DC000057FC15495E3108463E38FAF751FC124977
:10DC1000A03108468038FAF74BFC0F48002420302A
:10DC2000FAF7CAFB0C4AC1B24800A932801C107036
:10DC300003205070022000231546893D08E02E5D28
:10DC40001654401CC0B21354401C641CC0B2E4B251
:10DC50008C42F4D370BD000000F4FF1F54F0FF1F8E
:10DC6000303030300000000010B5134C2078002810
:10DC700006D0612211A10020FEF7F4FC022010BDA5
:10DC8000002211461046FBF7D7FC002801D01A20CD
:10DC900010BD00206070A070E070A060E060207196
:10DCA000206160610121A06189021248FAF7BDFC80
:10DCB00001202070002010BDD0F0FF1F2E2E5C2E02
:10DCC0002E5C2E2E5C736F757263655C6461706C84
:10DCD000696E6B5C647261672D6E2D64726F705C2F
:10DCE0006961705F666C6173685F696E74662E63EC
:10DCF0000000000088FFFF1F30B5002305E0DD00B5
:10DD00000C46EC40C4545B1CDBB29342F7D330BDED
:10DD1000F7B504462F481F250078AD0282B017469C
:10DD2000012808D0FF2279322BA10020FEF79AFCAF
:10DD3000022005B0F0BDAC4201D31F20F9E7FFF788
:10DD40001AF8002844D02E1B301FB84201D93A4699
:10DD500000E0321F1F4803998069FEF7A1FF1D49AB
:10DD60008861009001208002844207D228483A4608
:10DD700000190399FAF7A8FB0020DAE7E019A84296
:10DD800026D103988519281FFAF753FC0102203D7C
:10DD9000E87F090A0006014300980E4D884201D031
:10DDA0002320C6E739462046039AFFF7E7FD0028FF
:10DDB00001D01C20BDE70122920215490020FEF788
:10DDC00097FF0446FFF77EFE012068702046B0E70B
:10DDD0002220AEE7D0F0FF1F2E2E5C2E2E5C2E2EC2
:10DDE0005C736F757263655C6461706C696E6B5CAB
:10DDF000647261672D6E2D64726F705C6961705F13
:10DE0000666C6173685F696E74662E630000000063
:10DE100088FFFF1F10B5114904461F2009788002B2
:10DE2000012907D0FF22BB320DA10020FEF71AFC0A
:10DE3000022010BD844201D31F2010BDFEF79BFFBE
:10DE4000002801D0002C01D0222010BDFF22013279
:10DE50000020D101FEF74CFF10BD0000D0F0FF1FE5
:10DE60002E2E5C2E2E5C2E2E5C736F757263655C9D
:10DE70006461706C696E6B5C647261672D6E2D6499
:10DE8000726F705C6961705F666C6173685F696E08
:10DE900074662E630000000002468800064910B533
:10DEA00040188038C06F002804D0114601F0F8F8FF
:10DEB00001F0E6F810BD000044FAFF1F80B5012014
:10DEC0000649C0038860FAF745F9084F044A054936
:10DED0000548BC4600DF002080BD000000ED00E0EA
:10DEE00098F5FF1F0A20030055DF00007DF20000B7
:10DEF000024901224A7008717047000060F0FF1F5C
:10DF0000024901220A70C8707047000060F0FF1FCC
:10DF1000024901228A7048717047000060F0FF1FBB
:10DF200080B50448044F81680120C002BC4600DF70
:10DF300080BD000060F0FF1F7DEC000080B503484D
:10DF4000034F81680420BC4600DF80BD60F0FF1FE6
:10DF50007DEC00001FB50120064605460090162006
:10DF6000019000200290FEF73DFDFEF79DFB854FDE
:10DF7000BC4600DF844CA060FFF726FD0098FFF749
:10DF80006FFD3046FFF762FD2846FFF773FDFBF794
:10DF900063F900F07DFA00F081FAFFF71BFE03F051
:10DFA0001DF8012003F036FB002002F023FF0120C2
:10DFB000E0710B20784F03900023744A7449754830
:10DFC000BC4600DF774F002274497548BC4600DF2D
:10DFD000754FBC4600DF0446800509D56A48807944
:10DFE000002803D0714F0120BC4600DFFCF7FAFE89
:10DFF000600702D5022002F0CFF9E00612D5032017
:10E0000002F0CAF90020FFF71FFD002002F0F2FE27
:10E010000020FFF725FD0020FFF718FD0020FFF787
:10E0200029FDFEE7A00602D5032002F0B5F9200580
:10E0300001D5FEF76BFBE00735D05A2003F024FB37
:10E04000514FF87900282ED001280BD0032817D083
:10E05000052828D10020F871FFF7F6FC002002F017
:10E06000C9FE20E00398002802D0401E03901AD178
:10E07000012002F0BFFE0320F8711620019012E08B
:10E0800002F0B0FE002805D00120FFF7DDFC0220E1
:10E09000F87108E00198002802D0401E019002D1DA
:10E0A0000120FFF7D1FCA0078CD50298002804D0EE
:10E0B000FFF780FC002809D00DE0FFF77BFC00286B
:10E0C00009D0002002F068F9012003E0022002F0EC
:10E0D00063F9002002902C4C207800280BD0E078C7
:10E0E000012826D0022824D0012000900020207092
:10E0F0000098FFF7B5FCA07800280AD060790128C5
:10E1000026D0022824D001250020A0702846FFF741
:10E11000B1FC6078002800D154E72079012824D090
:10E12000022822D00126002060703046FFF78EFCC6
:10E1300048E70099012901D0012100E00021009168
:10E140000029D5D00128D3D100202070E070CFE77E
:10E15000012D01D0012500E00025002DD6D0012899
:10E16000D4D10020A0706071D0E7012E01D001262B
:10E1700000E00026002ED8D00128D6D10020607003
:10E180002071D2E7B9F4000060F0FF1F10F5FF1F07
:10E190000B880000B50301003DF40000FFFF000004
:10E1A000370A0000D9EC000025EC000019EC000053
:10E1B000014988717047000060F0FF1F10B5FFF73C
:10E1C0007FF910BD10B5FF2104460231FAF72DFA90
:10E1D00000F082FC00202070FFF772F910BD0000F3
:10E1E000012805D0022805D003280BD0CF2202E059
:10E1F000C32200E0C72204A10020FEF733FAFBF798
:10E200005BFDFEE7CB22F6E72E2E5C2E2E5C2E2E3B
:10E210005C736F757263655C6461706C696E6B5C76
:10E220005254585F436F6E6669672E6300000000AA
:10E23000FEE700000748016807484161002181614D
:10E24000072101610548016AFF221206114301629C
:10E2500040177047F41E010000E000E000ED00E010
:10E2600070477047FFB583B0054604980E9C281888
:10E2700000900020844F2060F878844E00281BD046
:10E280000020F870701E0278011D0698FAF71CF93C
:10E29000701E0078069941180691216808182060C0
:10E2A000786871783278000C090200041143084341
:10E2B000711E097840187860CAE028780A2813D0BF
:10E2C0000D2811D03A287DD0397800297BD0FEF76F
:10E2D00049FD02076D497878491E0B5C120F1A43FD
:10E2E0000A54401C7870ADE0684A0021521E137831
:10E2F00008465B1D9C4604E0135C5918401CC9B2DB
:10E30000C0B28445F8D8002901D00426A5E0B87829
:10E31000002844D10120B870707831780002084399
:10E3200040BA3070010A717001905848401EC078A0
:10E33000002806D0012833D0022833D004282ED15B
:10E340004EE052492522491E8818FAF7BDF8786830
:10E35000019A010C09041143814203D00120F87095
:10E3600002267AE04948401E0278011D0698FAF715
:10E37000ABF846480699401E00784118069121687E
:10E3800008182060786871783278000C090200045F
:10E39000114308433D49491E09784018786056E00A
:10E3A00001265AE021680C98FF22411A0698FAF7D4
:10E3B00017F920687968091A0D9801600098411BC7
:10E3C000049801E02AE033E0411A059801602F48E3
:10E3D000401E0179407909030001014379601AE088
:10E3E00021680C98FF22411A0698FAF7F9F820687C
:10E3F0007968091A0D9801600098411B0498411A28
:10E40000059801602148401E4179027908021043B5
:10E4100040BA00047860022007B0F0BD1B482521F7
:10E42000401EFAF702F9002038707870B8700EE0DC
:10E430007978252925D2FEF795FC144900017A78D0
:10E44000491E8854387800281BD0002038706D1C75
:10E450000098854200D030E7002621680C98FF2202
:10E46000411A0698FAF7BCF820687968091A0D98DD
:10E4700001600098411B0498411A059801603046DC
:10E48000CAE70120E2E70000ECF0FF1F890300204B
:10E4900000B500F003F901F019F800BD7047000065
:10E4A00070B5134D0646EFF31080C407E40F72B643
:10E4B0002846FAF707FF002C00D162B6002816D1D3
:10E4C000FF2210210B48FAF78BF809223146094840
:10E4D000F9F7FAFFEFF31080C407E40F72B6054AAC
:10E4E00010212846FBF7E4F8002C00D162B670BD7D
:10E4F00000FC010070200020F7B504461F2084B006
:10E500008002434F029038781646012805D0A12298
:10E5100040A10020FEF7A6F841E0FF21013188006C
:10E52000009001912046FAF79DF80225002901D0BC
:10E53000AA222FE00198864205D301463046FAF719
:10E5400091F8002901D0B12224E020460099FAF781
:10E5500089F800988919814201D9B8221AE0B8785F
:10E5600000280DD1F878002808D0B9688C4203D370
:10E57000F8680818A04203D8C6220BE0C02209E0C0
:10E580003979384600290DD07A6939698918A1424C
:10E5900008D0CE221FA10020FEF764F83D700220B3
:10E5A00007B0F0BD7F218902A7198C4205D2012155
:10E5B000C9038F4201D9002100E00121002910D0B8
:10E5C00013480121017146610461324620460599D4
:10E5D000FFF79EFB222807D00028E1D00C490D70E0
:10E5E000DEE705701C20DBE731462046059AFFF781
:10E5F000C5F9002801D00648F3E70298874204D302
:10E60000FFF760FA0249012048700020C8E70000C7
:10E61000D0F0FF1F2E2E5C2E2E5C2E2E5C736F759D
:10E620007263655C6461706C696E6B5C6472616777
:10E630002D6E2D64726F705C6961705F666C6173C2
:10E64000685F696E74662E6300000000FF20013071
:10E650007047EFF31082D207D20F72B603680B40F7
:10E660000360002A00D162B67047EFF31082D20730
:10E67000D20F72B603680B430360002A00D162B662
:10E680007047EFF31082D207D20F72B603684B4087
:10E690000360002A00D162B67047000008B5FF2071
:10E6A000094A033010600949486940084000486140
:10E6B00007480090401E0090FCD10869C007C00FB9
:10E6C0000021116008BD000000A0044040F00F4090
:10E6D00010270000F7B50446801801214002890286
:10E6E000884206D9124A13A10020FDF7BBFF002083
:10E6F000FEBD560231460198F9F797FF640265099D
:10E70000102D12D201277F02BC4201D2012000E06D
:10E7100000209122920007A1FDF7A4FF1249680191
:10E7200041183A1B0198F9F7CFFE3046FEBD0000B4
:10E730003A0200002E2E5C2E2E5C2E2E5C736F751E
:10E740007263655C6461706C696E6B5C6472616756
:10E750002D6E2D64726F705C7669727475616C5F7A
:10E7600066732E63000000000C11002010B5012418
:10E7700064020B46002801D0002010BD2246034948
:10E780001846F9F7A1FE204610BD00004C0A0020F3
:10E79000F8B50C46002801D00020F8BD204F38788D
:10E7A000012838D0022838D0002508461DA102F0E3
:10E7B000C5FC0646A0191EA102F0C0FC8619A019CE
:10E7C0001D4902F0BBFC8619A0191CA102F0B6FC81
:10E7D0008619A0191AA102F0B1FC8619A01979882E
:10E7E00002F0B5FC8619A01914A102F0A7FC861945
:10E7F000002D0ED0A01914A102F0A0FC8619A019BA
:10E80000294602F09BFC851960190CA102F096FCC8
:10E8100046193046F8BD0FA5C7E711A5C5E70000AA
:10E8200000F1FF1F4173736572740D0A0000000050
:10E8300046696C653A200000080800200D0A0000B7
:10E840004C696E653A200000536F757263653A201B
:10E8500000000000426F6F746C6F616465720000AD
:10E860004170706C69636174696F6E0010B50A461F
:10E87000002801D0002010BD01214902104602F0FD
:10E88000A3F810BDF8B50D46044602F0F5FE0646A5
:10E89000FEF73EFB07463046FEF75EFB0646002CC1
:10E8A00001D00020F8BD28461B4902F047FC044671
:10E8B0002819394602F042FC0419281917A102F060
:10E8C0003DFC154904192819C91F02F037FC041929
:10E8D00000270120009014E00098002804D1281996
:10E8E0000FA102F02BFC0419F00708D00D49B80065
:10E8F0000958281902F022FC04190020009076081B
:10E900007F1C002E01D0052FE6D3281903A102F0A9
:10E9100015FC0019F8BD0000931F01000D0A00004E
:10E920002C2000009C20010070B50C46002801D06E
:10E93000002070BD01256D0229462046F9F775FEBD
:10E940000648F9F739FD024604492046F9F7BCFDAF
:10E9500029462046FEF70AFB70BD00009B1F010000
:10E96000F8B5094D06460F462846F9F725FD044639
:10E97000002E01D00020F8BD024629463846F9F79E
:10E98000A3FD2046F8BD0000642F010010B501244E
:10E9900064020B46002801D0002010BD2246034926
:10E9A0001846F9F791FD204610BD00004C080020E4
:10E9B00004490A6A0260CA6942608969816000216B
:10E9C000C16070474080044010B50846540221469B
:10E9D000F9F72BFE204610BD70B5234D0024687852
:10E9E000A978E443884201D0012000E00020FF2202
:10E9F000F2321EA1FDF736FE6878022804D0002806
:10EA000016D0012818D020E02548FF240078F534DE
:10EA100000281AD0012809D0022816D0032814D0C3
:10EA2000204A12A10020FDF71DFE0EE01E4C0CE056
:10EA3000A878022808D008E0A878022802D0002888
:10EA400002D002E0194C00E00024601C05D1154AF8
:10EA500006A11032FDF706FE0024A868A04201D9E5
:10EA6000012070BD002070BDF4F0FF1F2E2E5C2E23
:10EA70002E5C2E2E5C736F757263655C6461706CC6
:10EA8000696E6B5C647261672D6E2D64726F705C71
:10EA90007666735F6D616E616765722E630000005C
:10EAA000F405002003020000204E0000C40900000D
:10EAB00070B5034600200246012509E0DC0704D0BA
:10EAC0008E1A2C46761EB44020435B08521CD2B2EC
:10EAD0008A42F3D370BD000010B525210748F9F72D
:10EAE000A4FD064825212530F9F79FFD04480021A3
:10EAF0004160017041708170C17010BD88030020B9
:10EB0000ECF0FF1F0146EFF31080C207D20F72B680
:10EB10000868002801D003680B60002A00D162B6A3
:10EB20007047000070B50D4600280FD00849094C09
:10EB3000884204D222680146104600F0D1FA2068CB
:10EB40004570054800F0FBF800F090FB70BD000038
:10EB5000FFFF0000A0F1FF1FB81F0020704700005A
:10EB600070B51B4EF068002831D0B08A401EB082CC
:10EB7000002526E0A068002808D061684160606830
:10EB8000002802D0A16881606560A5601048214618
:10EB9000183800F0CDFAA08AB0826078042804D139
:10EBA0000C49E08A09884018A08201206070202169
:10EBB0000855E068F060E068002801D00661E56073
:10EBC0002561B08A002802D1F468002CD2D170BD32
:10EBD000D01F0020A8F1FF1F70B504000ED00C4D0F
:10EBE000A17828680126827891420BD900F0BEFAFC
:10EBF00028684670204600F039FB70BD054800F0DB
:10EC00009EF8F8E766702146024800F091FA70BD60
:10EC1000A0F1FF1FB81F002010B50321FFF782FFEE
:10EC200010BD000001480068408B7047A0F1FF1F35
:10EC300010B50446008B084320836278618B062A56
:10EC400015D0052A12D1084210D00A46024062832C
:10EC500088432083204600F0ABFA01206070022137
:10EC6000202001552146044800F062FA10BD0A46F2
:10EC70008243EDD010BD0000B81F0020024688007E
:10EC800070B5144940188038C46F002C1DD0208BFB
:10EC9000104320836178658B062917D0052914D18C
:10ECA000284212D0294601406183A8432083204690
:10ECB00000F07EFA208B0221A8432083012060709F
:10ECC000202001552046FFF787FF70BD294681436C
:10ECD000EBD070BD44FAFF1F70B503460D480D46DA
:10ECE0000468002A208B08D01946814301D00621F0
:10ECF00009E098432083022070BD0146194001D0ED
:10ED00006183F6E7052163832846FFF70BFF0120A7
:10ED100070BD0000A0F1FF1F814202D342688A4209
:10ED200001D801207047EFF31082D207D20F72B6DC
:10ED300003680B60016000D162B600207047014695
:10ED40004068002342684A600A78022A05D0012AF6
:10ED500003D0032A01D0436070474268002A01D0E3
:10ED6000916043608360704770B50446154600208B
:10ED7000207001226270A1706060A060E06020617C
:10ED8000A082E0822083234660832033187058706D
:10ED9000608C002803D10448FFF7B4FEA062294626
:10EDA000204600F005F870BD88F9FF1F704700008D
:10EDB00030B5428C920803D10E4A12881204920C8C
:10EDC000836A92009B185A0700D51B1F0122120666
:10EDD000403BDA630022996314469500521C5C5153
:10EDE0000E2AFAD3C2691A624362C162806A02497A
:10EDF000016030BDF01E0100A52E5AE20349044A0D
:10EE00000968C8821288801888827047A0F1FF1FA5
:10EE1000A8F1FF1F10B50848016808488A8A0088D1
:10EE2000CB8A101AD21880B28A82010402D404213B
:10EE3000FFF778FE10BD0000A0F1FF1FA8F1FF1F33
:10EE4000F8B50446406800260F46002805D06078D3
:10EE5000022818D0A08900282FD0A089E1898842F3
:10EE60003ED2208980000019076172B6A089401C3B
:10EE7000A08162B62089401C80B22081E18988424D
:10EE800000D12681F8BD66702046FFF758FF054681
:10EE9000203006702189E86989000919086172B675
:10EEA000A089401CA08162B62089401C80B22081CC
:10EEB000E18988420AD1268108E02046FFF73FFF1A
:10EEC0000546C06904210760202041550120687073
:10EED000284600F06DF92946034800F029F9F8BDED
:10EEE0000320FFF77DF9F8BDB81F00200321017052
:10EEF000002141704180416081607047F8B504464F
:10EF00004088002804D0254EA1683268914201D083
:10EF1000FF20F8BD401E0004000C60803CD1316829
:10EF20006078887061680127002928D02046FFF7A3
:10EF300006FF0546052120300170284600F038F90B
:10EF40006780A560A87860701548316840688A7845
:10EF50008078824201D328460AE0114800F0E8F8A0
:10EF600029460F4800F0E4F8306847706F7011E0F0
:10EF7000FFF732FE31680020203108700CE00849AC
:10EF800049688A783168824206D9054800F0D0F88D
:10EF9000306847700020EBE70020F8BDA0F1FF1FAC
:10EFA000B81F002070B50E46184D044641882868E9
:10EFB000002907D0A168814208D16088401C608088
:10EFC000002070BDA06080786070F6E7002E0FD042
:10EFD00062788078824203D28870A06800F0D0F80E
:10EFE0006068002806D02046296800F0A1F808E0F3
:10EFF000012070BD2868606029680020486028688A
:10F00000846009213046FFF78DFDF1E7A0F1FF1F75
:10F0100070B51848012102685170006800F0A6F828
:10F02000154D6C7813E0E000411948680278002A19
:10F0300017D0012A1AD000F0EBF8E878641C84425B
:10F0400000D1002472B6A878401EA87062B6A878D5
:10F050000028E8D16C700948FFF771FE00F006F94E
:10F0600070BD098989B2FFF7E3FDE6E78968FFF71C
:10F07000E7FEE2E7A0F1FF1F20FAFF1FB81F002004
:10F0800005480178002902D0012141707047012014
:10F09000024900074860704798F1FF1F00ED00E04B
:10F0A000F8B50E4EF778B41C354672B6B278BA424F
:10F0B00007D2521C22702A78531CBB4200D1002375
:10F0C0002B7062B6F378934204D9D2009219916002
:10F0D0005060F8BD0220FFF783F8F8BD20FAFF1F4B
:10F0E00010B5124AD368002B17D013469B8A04E050
:10F0F000002C12D02246A48AE318D4688B42F7D39E
:10F10000C460D0600261C468002C00D02061591A2C
:10F110008182908A401A908210BD0024C460D06021
:10F12000C91A02619182848210BD0000D01F0020A4
:10F1300030B502780023022A03D0012A01D0032A25
:10F1400000D101238C7800E010464268002A02D0EA
:10F150009578A542F8D24A604160002B04D0002A7D
:10F1600000D09160886030BD0020FBE703494A6809
:10F17000426000228260486070470000B81F002093
:10F1800010B583680446002B05D1607801280CD1A6
:10F19000064B03E09B6818780028FBD0204600F05F
:10F1A0001DF821461846FFF7C3FF10BDB81F002009
:10F1B00010B5016900290FD0C268CA60C368002277
:10F1C000002B07D08B8A848A1B198B82C368196134
:10F1D000C26000E08A82026110BD000081680029DF
:10F1E00007D042684A604168002901D08068886081
:10F1F0007047064906E04A68824202D1406848608A
:10F20000704711460029F6D170470000B81F002052
:10F2100010B5416800290ED0FFF791FD0446FFF7B5
:10F22000C7FF0120607003212020015521460448BA
:10F23000FFF77EFF10BD4188491C418010BD0000D2
:10F24000B81F002010B507480068416A806A8142F3
:10F2500003D300680449884202D00120FEF7C0FFB2
:10F2600010BD0000A0F1FF1FA52E5AE20249486020
:10F270000221417070470000A0F1FF1FF7B515464D
:10F28000394A002004463749128802E08300CC50F6
:10F29000401C9042FAD33548302201883448FDF7AB
:10F2A0009EF9344801210088C90780B242183248CB
:10F2B00001683248FDF793F9314808220188314846
:10F2C0000068FDF78CF9304FFF26FE707C842F4AD2
:10F2D00000213846FFF748FD2D48042101704460A5
:10F2E0002C480170C46004618482786A2030F8F789
:10F2F0002BFF29482A4907600220787027480470AC
:10F3000044700978C170FFF751FD2648016A320444
:10F3100011430162C169026A5202920E92061143C0
:10F32000C161FEF787FF20490028086012DB8208D0
:10F330001E49920051180A688307DB0E9E40324333
:10F340000A60C206D20E012191404011184A800085
:10F350008018016000232A460199009800F06EF899
:10F36000FEBD000044FAFF1FEC1E0100041F010057
:10F37000B8F8FF1FF01E0100081F010088F9FF1FE9
:10F380000E1F01006CF0FF1FE81F002031E200009B
:10F39000B81F0020D01F0020A0F1FF1F20FAFF1F80
:10F3A0000C1F010000ED00E09CF1FF1F00E400E0F5
:10F3B00000E100E010B50B480121026851700068BF
:10F3C000FFF7D4FEFFF7CAFB07480168491C01603C
:10F3D000FFF7C6FB00F012F80448FFF7B0FCFFF798
:10F3E00045FF10BDA0F1FF1FA8F1FF1FB81F0020AF
:10F3F0000148006870470000A8F1FF1F70B50D4D6F
:10F400002868002815D0A8880B4E401EA8800AE066
:10F41000E088FEF726FFA088A880206828602146A3
:10F420003068FFF779FCA888002802D12C68002CEE
:10F43000EED170BDACF1FF1F6CF0FF1FFFB50806E9
:10F4400081B01E4617460C46000E00D14C1C1648D3
:10F45000FFF758FB051E25D02002000CAF62688420
:10F46000EE61E1B22846019AFFF77EFC10480124C4
:10F470000E49028806E0A00040188038C06F0028BE
:10F4800003D0641C9442F6D90024A00040188038B0
:10F49000C567EC702846FFF79FFB064800682030E0
:10F4A0000470204605B0F0BDB8F8FF1F44FAFF1FF6
:10F4B000EC1E0100A0F1FF1F02480068002800D0E8
:10F4C000C0787047A0F1FF1F00207047044A05492B
:10F4D000002801D0506800E0106808607047000004
:10F4E000441E010000F0FF1F10B5064C6078002894
:10F4F00007D10122520204490448F8F7E9FE01202D
:10F50000607010BD08F1FF1F0C0D00200C110020D1
:10F51000F8B50024274825460460047126462121B9
:10F520002548F9F782F8244821212130F9F77DF8A0
:10F53000214809214230F9F77AF81F4F1E48A100EF
:10F540005E384158781901F0D3FD4019641CE4B2CB
:10F55000C5B2042CF2D37E550025174F2C46213717
:10F560001548A1004E384158781901F0C1FD4019E5
:10F57000641CE4B2C5B2042CF2D30F4C0D497E5585
:10F58000423414392046096801F0B2FDC0B2265455
:10F590000A48042201680748F8F796FF0548302119
:10F5A0000671401D01703222427035228270C17096
:10F5B0000671F8BD54F0FF1F5EF4FF1F00F0FF1F3F
:10F5C000F1B5354DA8694169009888470746A86993
:10F5D0008169009888470446002F07D0002C05D089
:10F5E0000126B602B74209D8012008E0FF222632E0
:10F5F0002AA10020FDF736F80220F8BD0020FF22E6
:10F600002B3226A1FDF72EF839463046F9F72AF8B5
:10F61000002909D00020FF222C3220A1FDF722F87A
:10F62000BC4203D3012002E00120F4E70020FF22C6
:10F630002D321AA1FDF716F839462046F9F712F8CF
:10F6400000291FD00020FF222E3214A1FDF70AF856
:10F6500021460098F9F706F80098401AE8602C61F6
:10F660006860B44200D33446AC60297800290BD0DE
:10F67000A969C9688847040006D0A869406880471E
:10F680002046F8BD0120DEE7FF221148A968F8F7FF
:10F69000A7FF0020F8BD0000B4F0FF1F2E2E5C2E47
:10F6A0002E5C2E2E5C736F757263655C6461706C8A
:10F6B000696E6B5C647261672D6E2D64726F705C35
:10F6C000666C6173685F6D616E616765722E630061
:10F6D00088FBFF1F10B50A4C2078002808D000F0E6
:10F6E0008DF86068C168074888470021217010BD07
:10F6F000C12205A10020FCF7B5FF022010BD0000CB
:10F7000078F0FF1F54FAFF1F2E2E5C2E2E5C2E2E3B
:10F710005C736F757263655C6461706C696E6B5C61
:10F72000647261672D6E2D64726F705C66696C65C2
:10F730005F73747265616D2E63000000B0B5144C88
:10F7400005462078002801D0862202E0022D06D34B
:10F750008C2210A10020FCF785FF0220B0BD1A4FBB
:10F76000BC4600DFFF21A06005311848F8F75FFFB5
:10F7700001200749207028010C3140186060416861
:10F78000124888470028E9D003212170B0BD00004D
:10F7900078F0FF1F2E2E5C2E2E5C2E2E5C736F7564
:10F7A0007263655C6461706C696E6B5C64726167E6
:10F7B0002D6E2D64726F705C66696C655F73747218
:10F7C00065616D2E63000000B9F4000054FAFF1F5C
:10F7D000F8B5094D0E460746002420012A58314647
:10F7E00038469047002801D02046F8BD641CE4B29A
:10F7F000022CF2D30320F8BD84F0FF1F80B5074F21
:10F80000BC4600DF06498968884201D1012000E03A
:10F810000020632203A1FCF725FF80BDB9F400009E
:10F8200078F0FF1F2E2E5C2E2E5C2E2E5C736F75D3
:10F830007263655C6461706C696E6B5C6472616755
:10F840002D6E2D64726F705C66696C655F73747287
:10F8500065616D2E63000000014610B5083103227A
:10F860000C4608A0F8F7D4FD002807D00322214653
:10F8700005A0F8F7CDFD002801D0032010BD012020
:10F8800010BD000042494E004845580070B5154D66
:10F89000064628780C46012806D0A52212A1002091
:10F8A000FCF7E0FE022070BDFFF7A8FF6868224663
:10F8B00083683146194898470446102807D0112C10
:10F8C00007D0002C05D003202870204670BD0220F0
:10F8D000FAE72878012800D00020B32202A1FCF723
:10F8E000C1FEF2E778F0FF1F2E2E5C2E2E5C2E2E2E
:10F8F0005C736F757263655C6461706C696E6B5C80
:10F90000647261672D6E2D64726F705C66696C65E0
:10F910005F73747265616D2E6300000054FAFF1FFF
:10F92000F0B593B00F4604461E461546442168467E
:10F93000F8F77DFE189800950290199801960390AB
:10F9400060680990A0680D9020680E900120000664
:10F9500010900F97684600F03DFB002833D01C4DF7
:10F960001C4E002411A9304600F07EF9002829D051
:10F97000119880030AD5174800216F460C4664256C
:10F98000001D00F0BBFB00281CD003E0641CAC424F
:10F99000E8D317E03946304600F066F9002811D068
:10F9A0003868C00302D4641CAC42F3DBAC4209D01B
:10F9B00008483946083000F057F9002802D000986E
:10F9C000002802D0002013B0F0BD0120FBE70000AA
:10F9D00040420F00F0ED00E010B5F9F73DFC09489A
:10F9E00020214160402444608215426043690B43FA
:10F9F00043614169214341614169114341610120F2
:10FA000010BD000080F00F40F8B5002004460090C3
:10FA10002149401E086064254860FFF7DDFF00F0C3
:10FA2000BFFBF9F721FE002824D01E21002000F0A2
:10FA300013FB00281ED00021082000F00DFB002839
:10FA400018D005210907042000F006FB002811D07A
:10FA5000052676076946042000F0B0F8002809D092
:10FA600000993046884302D0641CAC42F2DBAC42C1
:10FA700001D10020F8BD0949042000F0EDFA00286A
:10FA8000F8D000F08DFC0021082000F0E5FA0028F5
:10FA9000F0D00120F8BD000070F0FF1F000F0050F3
:10FAA00007484169202291434161416940229143C5
:10FAB0004161416982159143416101207047000015
:10FAC00080F00F40F8B50D460446002A2CD0960869
:10FAD0001649002000F0C2F9002826D0052704228C
:10FAE00021466846FEF708F96946384600F0A6F94F
:10FAF000012819D10F270021384600F09FF901286D
:10FB000012D10024761E07E02946384600F096F907
:10FB1000012809D1641C2D1DB442F5D30E202946BD
:10FB200000F08CF9012800D00020F8BD520000231D
:10FB300038B50D4604460949002000F08FF9002829
:10FB40000BD06946204600F00BF8002805D0A0072E
:10FB5000C10E0098C8402870012038BD5000002315
:10FB60001CB50C460146042201A8FEF7C5F8052085
:10FB700001A900F063F901281ED10F20694600F0A9
:10FB80005DF9012818D10E20694600F057F90021CF
:10FB90006A462160D17809062160927812041143E7
:10FBA0006A4621605278120211436A462160127837
:10FBB00011432160012800D000201CBD38B50C463F
:10FBC0000C2108406946801C00F038F900216A4683
:10FBD0002160D178090621609278120411436A46A7
:10FBE00021605278120211436A4621601278114353
:10FBF0002160012800D0002038BDF8B514460F461A
:10FC0000054608E039462846FFF792FF002829D02C
:10FC1000641E6D1C7F1C002C23D0A807F2D112E0BB
:10FC2000A9050120890D8002461AB44201D2A60816
:10FC3000B600324639462846FFF744FF002811D067
:10FC4000AD19BF19A41B032CEAD808E03946284691
:10FC5000FFF76EFF002805D0641E6D1C7F1C002C72
:10FC6000F4D10120F8BD000070B50C4605460749E7
:10FC7000002000F0F3F8002806D021462846FFF7C0
:10FC80006FFF002800D0012070BD0000520000234B
:10FC90001CB500206A46FF211154401CC0B2082840
:10FCA000FAD311463320F9F795FF01201CBD00005F
:10FCB00070B520250B4C4026002810D0FFF7A4FE7D
:10FCC0000949042000F0CAF8002807D001210C20BF
:10FCD00000F0C4F8002801D0A560A66070BD656082
:10FCE000666070BD80F00F4044050040F8B50446E2
:10FCF000062801D0FFF770FE4C4E4D4DF11E23003B
:10FD0000FCF760FC070519095A5C768B920001200C
:10FD1000FFF7CEFF7FE00120FFF7CAFF454F02202B
:10FD2000BC4600DF0020FFF7C3FF0220BC4600DF17
:10FD3000FFF7B6FE6FE0FFF767FE00286CD0314694
:10FD4000284600F0DBF9002866D069462846FFF710
:10FD50008BFF002860D000988003F6D5344C012139
:10FD60000C34204600F0CAF9002855D0304E6946C0
:10FD7000E43E3046FFF778FF00284DD00098610D33
:10FD800008402D494118304600F0B8F9002843D00A
:10FD9000284F0220BC4600DF69462846FFF764FF73
:10FDA000002839D000988003F6D50021204600F0C5
:10FDB000A5F9002830D02EE02846F8E7F9F754FCE2
:10FDC000002829D01E21002000F046F9002823D069
:10FDD0000021082000F040F900281DD00521090766
:10FDE000042000F039F9002816D01049891EE3E7F5
:10FDF000FFF70AFE00280FD03146284600F07EF9B2
:10FE0000002809D069462846FFF72EFF002803D0B6
:10FE100000988003F6D50120F8BD284600F06EF961
:10FE20000028F9D0FFF73CFE0020F8BD03005FA0DA
:10FE3000F0ED00E019EC00000400FA0570B50D4685
:10FE40000646002429463046F9F752FC022803D121
:10FE5000641CE4B2642CF5D370BD000038B50D46C7
:10FE6000010E0446F022090610400143082000F06C
:10FE7000F3F8002806D0002C06D10E484168A942AC
:10FE800001D1012038BD45600C20044004222946E0
:10FE90006846641CFDF730FF69462046FFF7CEFF39
:10FEA000012805D10E200021FFF7C8FF0128E9D065
:10FEB000002038BD70F0FF1FF8B50D460446002A3B
:10FEC00025D0960813490020FFF7C8FF00281FD04F
:10FED0000527042221466846FDF70EFF694638468D
:10FEE000FFF7ACFF012812D10D27002407E02946B7
:10FEF0003846FFF7A3FF012809D1641C2D1DB44229
:10FF0000F5D30E200021FFF799FF012800D0002033
:10FF1000F8BD00005200002370B50C4605460849A4
:10FF20000020FFF79BFF002809D0A807C00E21463C
:10FF30008140284600F02EF8002800D0012070BD36
:10FF40005000002373B5064600246425104801992B
:10FF500000F0D4F8002815D00120000431460143F8
:10FF60000B48001F00F0CAF800280BD0084E083ECE
:10FF700001A93046FFF778FE002803D00198C0039E
:10FF800001D501207CBD641CAC42F1DB00207CBDAE
:10FF9000F8ED00E038B50C46014604226846FDF74E
:10FFA000ABFE05206946FFF749FF012810D1042266
:10FFB00021466846FDF7A0FE0D206946FFF73EFF8B
:10FFC000012805D10E200021FFF738FF012800D0BD
:10FFD000002038BD38B505460021082000F03CF867
:10FFE000002832D00024A00029582046FFF7AAFF9D
:10FFF00000282AD0641C042CF5D30920696AFFF775
:020000040001F9
:10000000A1FF002821D00D24A00029582046FFF789
:1000100099FF002819D0641C102CF5D31020296CEE
:10002000FFF790FF002810D009490A4800F066F851
:1000300000280AD069460420FFF7C0FD002804D03C
:100040000098A021084201D0002038BD012038BD11
:1000500001005FA0F0ED00E038B5082806D10B4A9A
:1000600013688B4201D1012038BD116004460C2277
:10007000144004226846FDF73FFE69462046FFF71C
:10008000DDFE0128F0D0002038BD000070F0FF1F19
:10009000F8B514460D46064608E029783046FFF7C5
:1000A0003BFF002829D0641E6D1C761C002C23D039
:1000B000B007F2D112E0B1050120890D8002471A84
:1000C000BC4201D2A708BF003A4629463046FFF796
:1000D000F3FE002811D0F619ED19E41B032CEAD821
:1000E00008E029783046FFF717FF002805D0641E86
:1000F0006D1C761C002CF4D10120F8BD70B50C46A7
:10010000054607490020FFF7A9FE002806D0214632
:100110002846FFF73FFF002800D0012070BD0000F7
:100120005200002380B5084FBC4600DF07494968EC
:10013000884201D1012000E00020FF22623204A1A8
:10014000FCF790FA80BD0000B9F40000F4F0FF1F46
:100150002E2E5C2E2E5C2E2E5C736F757263655C8A
:100160006461706C696E6B5C647261672D6E2D6486
:10017000726F705C7666735F6D616E616765722E1B
:100180006300000080B5054F02490348BC4600DF0C
:1001900080BD0000FFFF0000FC050020A5EF00006F
:1001A000704700007CB500250A4C2B46A0690095DD
:1001B000019581682A461830FFF7B2FB002807D066
:1001C000207F002802D000F03DF8054628467CBD7F
:1001D0000E207CBDB4F1FF1F7CB505460D48846937
:1001E000284600F019F801462846F8F73BFA00299E
:1001F0000DD1002000900190034620462A46183079
:10020000E168FFF78DFB002801D000207CBD0D20A8
:100210007CBD0000B4F1FF1F10B5094B596A0029DD
:100220000CDD491E0AD41A6ACC001459844203D842
:10023000C800001D105810BD491EF5D5186810BD26
:10024000B4F1FF1F7CB5114D0120AC6900F0A4F89A
:10025000002814D0E26A216BA06AFFF719FF00287A
:100260000FD000200090019003462046AA68183065
:100270002168FFF755FB002805D000207CBD072032
:100280007CBD08207CBD0A207CBD0000B4F1FF1FAE
:10029000F7B5324884B08569164605990498FFF78A
:1002A00013F9012833D10B2007B0F0BD6C6BB442B9
:1002B00000D934462246686A0599FFF7E9FE00280E
:1002C0003ED0686A00900027019728466B6B296929
:1002D0001830049A0290FFF723FB00282ED0FCF779
:1002E00071FB00280CD06969002933D0686A00903E
:1002F00023460197049A0298FFF712FB00281DD0AD
:1003000004980019049005980019361B0590002EDA
:10031000CCD10020C8E7102C01D2274600E01027DE
:100320003A4669460498FFF768FC002808D03A4628
:1003300069460598F8F712F8002803D00F20B3E7B4
:100340000920B1E70498F61BC01904900598C0195C
:10035000E41B0590002CDAD0DDE70000B4F1FF1FAC
:1003600070B5FF2405460134FFF756FFA04203D2C3
:100370002846FFF751FF0446204670BD10B5FCF734
:1003800019FB002801D0022000E0012000F004F851
:10039000FFF786FB002010BD10B5FFF7A7FC10BDCE
:1003A00001207047884203D3904201D80120704752
:1003B000002070470D4F00240320BC4600DF0C4D89
:1003C0000C4FBC4600DF0C4F0220BC46A96800DF82
:1003D00003212046F8F746F9641CE4B20029EFD166
:1003E0000120BC46A96800DFEAE70000FDED00003F
:1003F00060F0FF1F15EE00007DEC000080B5114895
:100400008078002807D00F48002120384A1E01605C
:100410008260816180BD0B4828220B492038F7F7A4
:1004200057FFFFF7AFFE09488178012903D14178D2
:10043000022900D181700348054F0830BC4600DF17
:1004400080BD0000F4050020641F0100F4F0FF1FD0
:10045000FDEE0000F8B51B4C1546E0780E4600286E
:1004600006D05722D20018A10020FCF7FBF8F8BDF7
:10047000E8051DD00020AF22920013A1FCF7F2F88E
:1004800060781E4A10A1FCF7EDF829463046FFF7C8
:10049000FDF90027012610280CD011280FD0277154
:1004A000084920394A6952194A6100F0CBF8F8BD71
:1004B0000120E0E7FFF70EF96770E67000E000202A
:1004C0002671EDE7F40500202E2E5C2E2E5C2E2EDC
:1004D0005C736F757263655C6461706C696E6B5C94
:1004E000647261672D6E2D64726F705C7666735FE7
:1004F0006D616E616765722E63000000BD020000D1
:10050000F8B51A4C074660780D46002812D0002036
:10051000174A18A1FCF7A6F8681C00D00120144A5D
:1005200014A1521CFCF79EF8104E203E7068401C2F
:1005300002D002E00120EBE77560E079032800D1EA
:10054000E7717068A84202D1E079B84201D0032077
:1005500008E03846FFF7F2F8002803D10121F560E2
:100560006170A17000F06EF8F8BD0000F405002085
:100570007D0200002E2E5C2E2E5C2E2E5C736F757D
:100580007263655C6461706C696E6B5C64726167F8
:100590002D6E2D64726F705C7666735F6D616E6137
:1005A0006765722E6300000070B5174C2578032D27
:1005B00005D02546203D2E68002E06D006E0134AC1
:1005C00013A10020FCF74EF870BD2860A868401CFD
:1005D00000D1A960E079032800D1E371A8699042B5
:1005E00004D9E869904201D9032009E0481C02D0EF
:1005F000A8688842F8D1E0799842F5D10020AA6134
:1006000000F020F870BD0000F40500202D0200006D
:100610002E2E5C2E2E5C2E2E5C736F757263655CC5
:100620006461706C696E6B5C647261672D6E2D64C1
:10063000726F705C7666735F6D616E616765722E56
:1006400063000000FEB50546102803D0112D01D02F
:10065000012000E00020464A46A1FCF703F8524C76
:100660002078032810D02246203A1168002912D0A1
:10067000D369906983420ED300280CD093685068E8
:10068000984208D1012007E0394A3AA1121D002002
:10069000FBF7E8FFFEBD00206071A37901930029FC
:1006A00002D1E179032901D0012100E0002100916C
:1006B000002804D02179002901D0012600E000267D
:1006C000E178002903D0002801D0012000E00020BB
:1006D000029010690027401C14D03348203840682D
:1006E000401C00D00120224A22A12232FBF7BAFF8F
:1006F0002D482038426801694069891A49028842B8
:1007000000D901270320002D01D020701DE00199A0
:1007100000290AD0002F01D00625F6E7009900290C
:10072000F3D0002EF1D10425EFE702990029ECD196
:10073000002E01D0022003E00098002802D0012002
:10074000207011E0207803280BD16078002806D0B3
:10075000FEF7C0FF00216170002D00D1054613484F
:1007600005700198002895D100F06EFFFEBD0000D5
:10077000DD0200002E2E5C2E2E5C2E2E5C736F751B
:100780007263655C6461706C696E6B5C64726167F6
:100790002D6E2D64726F705C7666735F6D616E6135
:1007A0006765722E63000000F4050020F4F0FF1F5F
:1007B00070B5012514486D0305601448826BC1149F
:1007C0000A438263426B0A434263114CE078F3218F
:1007D0000840E070E0785F210840E070FCF7AAF87C
:1007E0000D480C49C160C91E0161E0780C21084325
:1007F000E070E07820210843E07008480560024876
:1008000080380560012070BD80E100E00080044078
:1008100000B006400303000000B0044080E200E0A6
:100820000A4610B501460248FCF75AF810BD000010
:10083000DC15002010B50124074864030460074854
:10084000C1784906490EC170FCF774F80248803837
:100850000460012010BD000080E100E000B006400F
:10086000F8B5064600250120204940032F460860C0
:100870001F4CE0785F210840E070E078F3210840E9
:10088000E070FCF757F871790020012902D00229A5
:1008900003D004E001252F4600E0012501200001DE
:1008A000690008433843A0703068010111480068AE
:1008B000F7F7D8FE2178400849094901C204D20E51
:1008C0001143217061786070E0780C210843E0707A
:1008D0000120094940030860044980390860E07834
:1008E00020210843E0700120F8BD000080E100E015
:1008F00000B0064028F1FF1F80E200E070B50A4614
:1009000001460C48FCF701F80546EFF31080C407D8
:10091000E40F72B60748FBF74AFF002804D00648E8
:10092000C17880221143C170002C00D162B62846E4
:1009300070BD0000CC13002000B0064010B5024886
:10094000FBF724FF10BD0000CC13002010B50F4CA6
:100950002078002807D000202070FBF731FE002807
:1009600008D01B2010BD822209A10020FBF77AFECF
:10097000022010BD6078002803D1FCF7FAF90028A6
:1009800001D0002010BD212010BD0000D0F0FF1FBD
:100990002E2E5C2E2E5C2E2E5C736F757263655C42
:1009A0006461706C696E6B5C647261672D6E2D643E
:1009B000726F705C6961705F666C6173685F696EAD
:1009C00074662E6300000000F8B50F460446F7F782
:1009D0002CFE20468DA100F0B1FB0546601998A1C0
:1009E00000F0ACFB4519601999A100F0A7FB45196F
:1009F00060199BA100F0A2FB4519FBF7DBFF002863
:100A000001D09BA100E09BA1601900F097FB451964
:100A1000601999A100F092FB4519601997A100F0A7
:100A20008DFB4519FBF7CEFF002801D090A100E017
:100A300090A1601900F082FB451960198EA100F0A9
:100A40007DFB4519601993A100F078FB4519FBF770
:100A5000C1FF002801D086A100E086A1601900F046
:100A60006DFB4519601984A100F068FB4519FCF77E
:100A700080F9002801D08DA600E08FA6601991A111
:100A800000F05CFB45196019314600F057FB451931
:100A9000601979A100F052FB45196019314600F048
:100AA0004DFB451960198BA100F048FB4519FCF777
:100AB00060F9002815D1FDF72FF8002811D0601932
:100AC00088A100F03BFB4519FDF738F80146601995
:100AD000042200F062FB4519601967A100F02EFBAB
:100AE0004519FCF748F9002815D1FDF743F800280F
:100AF00011D0601981A100F021FB4519FDF74CF8D8
:100B000001466019042200F048FB451960195AA1FA
:100B100000F014FB451960197DA100F00FFB451989
:100B200060197EA100F00AFB4519601952A100F07E
:100B300005FB4519601984A100F000FB45196019F7
:100B4000002100F004FB451960194BA100F0F6FAF2
:100B50004519601980A100F0F1FA4519601983A1C7
:100B600000F0ECFA4519601981A100F0E7FA451987
:100B7000601981A100F0E2FA4519601980A100F026
:100B8000DDFA451960193CA100F0D8FA4519FCF7C7
:100B9000C3FF002810D060197CA100F0CFFA4519DE
:100BA000FCF7D4FF0146601900F0A2FA451960195C
:100BB00031A100F0C3FA4519601979A100F0BEFA1D
:100BC0004519FCF7C9FF0146601900F091FA451973
:100BD000601929A100F0B2FA4519601975A100F059
:100BE000ADFA784945196019496800F0B0FA45191D
:100BF000601921A100F0A2FA4019201872A100F09A
:100C00009DFA39462046FCF7B1F9F8BD232044414E
:100C1000504C696E6B204669726D77617265202D4C
:100C2000207365652068747470733A2F2F6D626548
:100C3000642E636F6D2F6461706C696E6B0D0A00BA
:100C4000556E697175652049443A2040550D0A007A
:100C50004849432049443A2040440D0A000000001E
:100C60004175746F2052657365743A20000000006E
:100C700031000000300000000D0A00004175746F63
:100C80006D6174696F6E20616C6C6F7765643A207A
:100C9000000000004F766572666C6F7720646574A3
:100CA000656374696F6E3A2000000000426F6F74D4
:100CB0006C6F616465720000496E74657266616391
:100CC000650000004461706C696E6B204D6F646557
:100CD0003A2000002056657273696F6E3A204056C4
:100CE0000D0A0000426F6F746C6F6164657220566C
:100CF000657273696F6E3A2000000000496E74657A
:100D000072666163652056657273696F6E3A200082
:100D1000476974205348413A200000003638326455
:100D20003833303365333733353535333234303259
:100D300062386439336334663234306133636563F7
:100D400030326139000000004C6F63616C204D6FE0
:100D500064733A200000000055534220496E7465C8
:100D60007266616365733A20000000004D534400D1
:100D70002C204344430000002C204849440000003C
:100D80002C2057656255534200000000426F6F747B
:100D90006C6F61646572204352433A2030780000E2
:100DA000496E74657266616365204352433A203030
:100DB0007800000052656D6F756E7420636F756EFC
:100DC000743A200000F1FF1F55524C3A2040520D5A
:100DD0000A00000010B500F083F800F00DF9F9F7F3
:100DE00095F910BD02484078002800D001207047D6
:100DF0001CF2FF1F10B5F9F7BDFA10BD00207047B7
:100E000070B51546012820D1002B01D0012B1CD133
:100E10000F4CA168002914D0491EA16020690D491A
:100E20008001411840222846F7F74EFB2069052132
:100E3000401CF7F717FC21616068401C606040208F
:100E400070BD012B01D101202070002070BD000079
:100E500008F0FF1FC0F2FF1FF8B507461A481646F4
:100E60000088824201DD0020F8BD18480078002883
:100E7000FAD0174C0122E26001E0002814D0628809
:100E8000002AFAD1134D32462F70681CF7F71CFB6D
:100E9000204665610024848046800F490978012935
:100EA00008D86D1C456108E00020E0606061A0800A
:100EB0006080D8E74188491C41800020F9F780FD17
:100EC0000648C4550120F8BD542301001DF2FF1F40
:100ED00040F2FF1F2C1800205223010076F1FF1F63
:100EE000002104480122C1600161027005224260B4
:100EF0008160704708F0FF1F0178832902D1407894
:100F0000002801D000207047012070477047000082
:100F1000F8B501261746022823D1002B21D03878B6
:100F200007281BD01D4C606800282DD0401E606033
:100F3000E0681B4D800140191A463946F7F7C4FA9C
:100F4000E068800141193846F7F7DAFCE068800173
:100F50004019FFF7D1FF012804D004E01149012016
:100F60000870F8BD0026E0680521401CF7F77AFB01
:100F7000E160A068401CA0602078002809D0FCF740
:100F800083FD0020207004E0912207A10020FBF7E0
:100F900069FB3046FCF7B4FFF8BD000008F0FF1F06
:100FA000C0F2FF1F04F0FF1F2E2E5C2E2E5C2E2E93
:100FB0005C736F757263655C6461706C696E6B5CA9
:100FC000636D7369732D6461705C757362645F75C2
:100FD0007365725F6869642E6300000010B505498F
:100FE0000020C870FFF7F6FEFAF758FEF9F7C2FFC7
:100FF00010BD00001CF2FF1FB0B5094FBC4600DF5A
:10100000084C0A4F60600848BC4600DFFBF74EFB07
:1010100000206070A0700649A0600860B0BD0000AC
:10102000B9F40000F4F0FF1FFC050020EDEE000015
:1010300068F2FF1F70B514460D460646FFF772F8BA
:10104000064B1868002807D00120FCF761FF2246F4
:101050002946304600F096FB70BD000068F2FF1F85
:1010600070470000F8B515460E460746FFF75AF8D8
:101070000D480068002816D00C4900200C4C8860F0
:10108000207803280FD00120FCF742FF2A46314682
:10109000384600F029FD2078032804D02A4631463E
:1010A0003846FCF723F8F8BD68F2FF1FF4F0FF1F85
:1010B000F40500200548074A01780548C180002151
:1010C00001704170C1608260016170473E23010080
:1010D0001CF2FF1F0100010010B5EFF31080C407E0
:1010E000E40F72B6FBF7C6FC002C00D162B610BD4F
:1010F00070B50D460446090E00F014F806462802A5
:10110000010EA01900F00EF886192804010EA0198E
:1011100000F008F88619E9B2A01900F003F8801968
:1011200070BD00000B09044A0907D35C0370090F66
:10113000515C417002207047301F010003460020BF
:1011400001E01A54401C0A5C002AFAD17047F3B53A
:1011500081B0074600242546029805E00A21F7F7EA
:1011600081FA0021641C4D410028F7D12046284314
:1011700001D101240025002609E00A210298F7F791
:1011800071FAA21B3031521EB954761C0290002015
:10119000311BA841F1D32046FEBDF8B515460E46D9
:1011A0000746FFF7D4FF0446A8420AD23022294658
:1011B0003846F7F715FA281BC0193146FFF7C7FF65
:1011C0002846F8BDF8B505460020042400902246C4
:1011D00029466846F7F778F90C4E0098726931692C
:1011E000FFF7E0F800280FD0291904226846F7F726
:1011F0006BF9F268B1680098FFF7D4F8002803D0C3
:10120000241D0C2CF0D90120F8BD0000B4F1FF1F03
:1012100001783A290AD1007A302809D0322807D03B
:10122000332805D0342803D0352801D0002070475A
:1012300001207047FFB583B00398FBF793FFFF22AF
:10124000663241A1FBF70EFA4C480190417A007AD0
:10125000090201434948C01E407B4143069840189B
:10126000401EF7F7FFF9054606980027444E002870
:1012700019D00024681EF76800900AE0F168481C45
:1012800082B2404800F034FDF068401CF0600098E5
:10129000641C8442F2D33C4A3A48F16800F028FDCD
:1012A000F068401CF0603069202802D3FF227B32B6
:1012B0001FE04101354A401C8C183061202234491E
:1012C0002046F7F701F90B2220460399F7F7FCF8BF
:1012D00021461C310698F7F7BDF9380C2075000A35
:1012E0006075A776380AE076B168102908D3FF2226
:1012F000893215A10020FBF7B5F9002007B0F0BD39
:1013000008460C225043214A224BC03A1350224B2C
:1013100087187B60049B002B00D013500598002891
:1013200000D078600198491C427A037A1002134A6F
:101330001843D21E527B50436843B860B160307886
:10134000401C30702046D9E72E2E5C2E2E5C2E2EAF
:101350005C736F757263655C6461706C696E6B5C05
:10136000647261672D6E2D64726F705C7669727441
:1013700075616C5F66732E63000000004F080020EB
:1013800008F1FF1F4C0A0020FFFF00000C0D002099
:1013900000230100C9E90000251E0100C07A704742
:1013A00010B51C30F7F745F910BD000010B5044624
:1013B000FFF7F6FF002812D0E07EA17E0402094864
:1013C0000C43017BC07A0902014307484069F7F7E3
:1013D00049F90449A41E497B6143081810BD002047
:1013E000C04310BD4C08002008F1FF1FC1727047B8
:1013F00070B50F49087DCA7C0402087BC97A0502D2
:1014000014430D43002C01D06C430FE008482030FA
:10141000F7F70FF9002802D06843044606E00024DD
:10142000FF225A3203A12046FBF71CF9204670BD6B
:101430004C0800202E2E5C2E2E5C2E2E5C736F75B9
:101440007263655C6461706C696E6B5C6472616729
:101450002D6E2D64726F705C7669727475616C5F4D
:1014600066732E6300000000F3B501260F46760276
:1014700081B031465048F7F7DAF831464F48F7F770
:10148000D6F84F4C0025C0214E48E560F7F7CFF85D
:101490004C487100C030F7F7CAF831464A48F7F7B0
:1014A000C6F825612570A560484865616060657073
:1014B000324647494048F6F70BFF3F4E307BF27A01
:1014C00001020120000411433818F61CF7F7CAF88E
:1014D0000446F71E797B3F484843A04208D9FF22C3
:1014E00027323DA10020FBF7BDF87C7B39480BE09B
:1014F00046484143A14208D2FF222A3236A10020A9
:10150000FBF7B0F87C7B414844432B4901200004A1
:101510002031844204D33574280A7074204603E0D5
:101520003474200A70740020F7F794F8797B204611
:10153000F7F798F83549000211394018040CFC827D
:10154000302233491F48F6F7C3FE60021D491C4C88
:101550004861086204206561A06000200C224243BB
:10156000521892686369401CD21862610428F5D34E
:10157000264A294667321148E56000F0B9FBE16868
:10158000224A491C6E320D48E16000F0B1FBE06870
:1015900025610C4D401C1E49E060C03528462022C4
:1015A0003031F6F791FF28460B220199F6F78CFFB0
:1015B00001202061FEBD00004C0800204C0A0020E4
:1015C00008F1FF1F4C0C00200C11002055D000002A
:1015D000B02001005A1000002E2E5C2E2E5C2E2E04
:1015E0005C736F757263655C6461706C696E6B5C73
:1015F000647261672D6E2D64726F705C76697274AF
:1016000075616C5F66732E630000000091FF00003F
:10161000B0220100B0B50446FEF7B4FD0749002C26
:1016200009D08878002801D102208870054F04482D
:10163000BC4600DFB0BD0020F7E70000F4F0FF1F5C
:10164000FC050020FDEE000080B5FEF79BFDFBF7DA
:1016500091F8002805D105484178022901D10121DE
:101660008170044F0248BC4600DF80BDF4F0FF1FCC
:10167000FC050020FDEE000010B5FEF753FD01480B
:10168000007810BDF4F0FF1FF8B50646FEF74AFDDE
:10169000FEF778FDFBF76EF8002815D0FDF79CF9F2
:1016A000264C05462648A168814201D28819A060CF
:1016B000254F2448BC4600DF002D09D0A07866786D
:1016C0006070012807D104E01F4F1E48BC4600DFB0
:1016D000F8BD0221A17021461B4F04460025194880
:1016E000BC468D6000DF0127002E17D0012E15D0DB
:1016F000022E13D1134E083E3078032803D0B77161
:101700000020FEF79FFF3078032812D00020FF2230
:101710000A320EA1FAF7A6FF00F0E6F8184E002CE8
:1017200009D0012C07D0022CD2D1FAF7BFFF3760C5
:10173000F8BD0120EBE73560F8BD0000F4F0FF1FB5
:1017400060EA0000FC050020FDEE00002E2E5C2E5D
:101750002E5C2E2E5C736F757263655C6461706CB9
:10176000696E6B5C647261672D6E2D64726F705C64
:101770007666735F6D616E616765722E630000004F
:1017800068F2FF1FF7B582B00446154600265102E5
:101790000398F6F74AFF0027FDF7A6FE31460C2016
:1017A000104A414388188068400A38180190BC42AA
:1017B0000ED384420CD2001BA84200D328460090CE
:1017C0005358E01B009A03999847009824182D1A43
:1017D000002D04D0761CF6B2019F102EDED305B08A
:1017E000F0BD00004C0C002001494860704700002B
:1017F00008F1FF1F1CB5012189062848FFF734FEB8
:101800002748FCF7CFF80346002225492548FFF773
:1018100011FD2548FCF7C6F803460022224923A003
:10182000FFF708FDFFF728FF002808D02248FCF743
:10183000B9F803460022204920A0FFF7FBFC224B09
:1018400041219A1C2148FBF723F900280BD020489E
:10185000FCF7A8F8034600221D491E48FFF7EAFCE2
:101860000021FFF7C3FD002001900120C00300907C
:10187000FBF781FA002810D0FF220132009901986D
:10188000F6F76CFD002808D11348FCF78BF80346E7
:101890000022114911A0FFF7CDFC1CBD341E010030
:1018A00029E90000281E01006DE80000444554416C
:1018B000494C53205458540085E800004641494C97
:1018C000202020205458540000F1FF1F0808002059
:1018D00091E700008F20010061E900004E4545447A
:1018E0005F424C205458540010B5FBF742FA0028D0
:1018F00005D0FFF7C1FE002801D1F8F7DDF9FBF7AD
:101900003AFA002805D0FBF7FFF8002801D0F8F7D5
:10191000D3F902484168491C416010BD00F1FF1F26
:1019200070B50C460546FCF74DF8002803D1FCF7CE
:1019300041F8002801D0012200E00022002A03D152
:10194000FBF740F800280ED0002C0DD0012C0AD156
:101950000B223B492846F6F701FD002803D1FFF78B
:10196000BBFBFFF771FE70BD0B2236492846F6F728
:10197000F5FC002841D00B2233A12846F6F7EEFCF7
:10198000002842D00B2233A12846F6F7E7FC0028B6
:101990003CD00B2232A12846F6F7E0FC002838D0D4
:1019A0000B2232A12846F6F7D9FC0028D9D00B2209
:1019B00031A12846F6F7D2FC002830D00B2231A105
:1019C0002846F6F7CBFC00282AD00B2230A1284667
:1019D000F6F7C4FC002826D00B2230A12846F6F7E3
:1019E000BDFC00282AD00B222FA12846F6F7B6FC12
:1019F0000028B8D1FBF726F9B3E7FBF7BCF90028BC
:101A0000AFD00120FBF7B4F8ABE70120FBF706F9F4
:101A1000A7E79E2227A10020FAF724FE70BD01202F
:101A2000FBF706F99DE72F4C206800688047206887
:101A30000069804720684068804792E70120D9E725
:101A40008F200100511E01004155544F5F525354E5
:101A500043464700484152445F525354434647006F
:101A6000415353455254202041435400524546525D
:101A700045534820414354004155544F5F4F4E2039
:101A8000434647004155544F5F4F46464346470043
:101A90004552415345202020414354004F56464C67
:101AA0005F4F4E20434647004F56464C5F4F4646D9
:101AB000434647002E2E5C2E2E5C2E2E5C736F75D7
:101AC0007263655C6461706C696E6B5C64726167A3
:101AD0002D6E2D64726F705C7666735F75736572C0
:101AE0002E6300002C1F0100F7B5002782B01546B9
:101AF00004463E46FDF7F8FC1EE00C203946414303
:101B0000104809188868400A30180190B4420ED372
:101B100084420CD2001BA84200D3284600904B6898
:101B2000A01B009A03999847009824182D1A002D9D
:101B300006D07F1C019EFFB2034880688742DCD339
:101B400005B0F0BD4C0C002008F1FF1FF7B50546AD
:101B500004462035287C84B01646302801D3606BBB
:101B600032E030210F1AB74200D3174600193A4627
:101B70000599F6F7A9FC287CC019C1B2297430294F
:101B800002D2002007B0F0BD05980023C0190590CF
:101B9000F61B1A462046FBF7CBFB00281FD002A9F4
:101BA0000022009101AB1146FBF70EFC0028E9D1A1
:101BB000019860632A7C2146FBF7BCFC0028E1D138
:101BC000297C606B4018606332460599FBF7B2FCD4
:101BD0000028D7D1606B801960631120D2E71920EB
:101BE000D0E70000F7B58118012349029B0288B0B5
:101BF000994206D92E4A2FA10020FAF733FD0BB0E7
:101C0000F0BD41024B095102049149090691364940
:101C10005A0151180291039109990191002801D0AC
:101C200000263BE0012639E0019970014418039930
:101C300000904518202221462846F6F78FFB002801
:101C40002BD0214628460B22F6F788FB002811D01E
:101C50000020264F05907F6823462A462046022111
:101C6000B84701990098085CE52805D00598002838
:101C700007D012E00120ECE72A4623461046012156
:101C800008E02046FBF76EFA002806D023462A46D5
:101C900018460021154C6468A047761C06988642B9
:101CA000C2D3049A09990298F6F70EFCA7E7000040
:101CB000560200002E2E5C2E2E5C2E2E5C736F754D
:101CC0007263655C6461706C696E6B5C64726167A1
:101CD0002D6E2D64726F705C7669727475616C5FC5
:101CE00066732E63000000000C0D002008F1FF1F3A
:101CF00010B54B000124591C6402A14206D3FF22F7
:101D0000083204A10020FAF7ADFC10BDC254120A3B
:101D1000425410BD2E2E5C2E2E5C2E2E5C736F75E1
:101D20007263655C6461706C696E6B5C6472616740
:101D30002D6E2D64726F705C7669727475616C5F64
:101D400066732E6300000000F0B587B000241646CD
:101D50000F460546039404940594FF2004AA03A9A2
:101D600001300292019100906B1C05AA3146384661
:101D7000FCF778FA00280DD0022814D001281FD0D3
:101D8000042829D0052801D00628E6D1052825D029
:101D9000012024E0049A002A27D0691C0398FBF74D
:101DA000C9FB044621E0049A002A05D0691C039867
:101DB000FBF7C0FB040018D10598361A3F18CCE792
:101DC000049A002A04D0691C0398FBF7B3FB04466D
:101DD000002C0AD1102408E0122406E00020FF2283
:101DE000623203A1FAF73EFC1324204607B0F0BD8F
:101DF0002E2E5C2E2E5C2E2E5C736F757263655CCE
:101E00006461706C696E6B5C647261672D6E2D64C9
:101E1000726F705C66696C655F73747265616D2E5C
:101E200063000000704700004D4943524F4249543F
:101E300048544D004D4943524F4249542020200000
:101E400084270100AC270100B4270100312E313076
:101E50000053544152545F424C414354B02E010050
:101E6000542E0100342E0100E82E0100582B0100F1
:101E7000FC2D0100702B01004C2D0100EC2C010009
:101E8000A82D0100B02C0100102F01006C2E0100C4
:101E90000C2C0100E02B0100B82B0100882D010063
:101EA000CC2E010028290100E8280100AC280100FF
:101EB0003C2C0100242B0100802A0100482A01004B
:101EC000702901004C280100802801002028010011
:101ED000C0270100F0270100E02A0100C02901000D
:101EE000FC290100BC270100BC2A010004000000FD
:101EF00088000401FF5207000100000010270000C5
:101F000000000000CC000000980000000400000069
:101F1000450201007D03010091020100D901010089
:101F2000A50101006103010019020100101F010059
:101F3000303132333435363738396162636465663F
:101F40000000000069DC00004D090100F9E4000018
:101F500035CE00009DCD00004DE6000009CF000009
:101F6000441F010000000000FFFFFFFFFFFFFFFF15
:101F7000FFFFFFFFFFFFFFFF000000000000000069
:101F8000000000000000000000000003747970658C
:101F90003A20006572726F723A20003C21646F63D0
:101FA000747970652068746D6C3E0D0A3C212D2D8E
:101FB000206D62656420506C6174666F726D20578D
:101FC00065627369746520616E642041757468652B
:101FD0006E7469636174696F6E2053686F727463A5
:101FE0007574202D2D3E0D0A3C68746D6C3E0D0AF3
:101FF0003C686561643E0D0A3C6D657461206368F0
:1020000061727365743D227574662D38223E0D0A27
:102010003C7469746C653E6D6265642057656273DB
:102020006974652053686F72746375743C2F7469AA
:10203000746C653E0D0A3C2F686561643E0D0A3C78
:10204000626F64793E0D0A3C7363726970743E0D71
:102050000A77696E646F772E6C6F636174696F6E57
:102060002E7265706C6163652822405222293B0DF7
:102070000A3C2F7363726970743E0D0A3C2F626FC5
:1020800064793E0D0A3C2F68746D6C3E0D0A004168
:10209000535345525420205458540000DC2F010063
:1020A000F82F0100E82F0100F02F0100D02F0100D0
:1020B000EB3C904D53443053342E31000208010064
:1020C000022000501FF80100010001000000000084
:1020D00000000000000029741902274441504C49B7
:1020E0004E4B2D444E4446415431362020200000B2
:1020F00000000000000000000000000000000000E0
:1021000000000000000000000000000000000000CF
:1021100000000000000000000000000000000000BF
:1021200000000000000000000000000000000000AF
:10213000000000000000000000000000000000009F
:10214000000000000000000000000000000000008F
:10215000000000000000000000000000000000007F
:10216000000000000000000000000000000000006F
:10217000000000000000000000000000000000005F
:10218000000000000000000000000000000000004F
:10219000000000000000000000000000000000003F
:1021A000000000000000000000000000000000002F
:1021B000000000000000000000000000000000001F
:1021C000000000000000000000000000000000000F
:1021D00000000000000000000000000000000000FF
:1021E00000000000000000000000000000000000EF
:1021F00000000000000000000000000000000000DF
:1022000000000000000000000000000000000000CE
:1022100000000000000000000000000000000000BE
:1022200000000000000000000000000000000000AE
:10223000000000000000000000000000000000009E
:10224000000000000000000000000000000000008E
:10225000000000000000000000000000000000007E
:10226000000000000000000000000000000000006E
:10227000000000000000000000000000000000005E
:10228000000000000000000000000000000000004E
:10229000000000000000000000000000000000003E
:1022A000000000000000000000000000000000002E
:1022B0008DE90000251E0100000200006DE700000E
:1022C000251E0100000000006DE70000251E010032
:1022D00000000000D5E60000E51B0100000400003E
:1022E00000000000000000000000002800000000C6
:1022F000000000000000418EBB3200000000000022
:1023000000000000000000000000000100000000CC
:10231000764876480000DC83764800000000000024
:10232000080010001800200030004000600080000D
:10233000C00000018001000200030004000600004C
:1023400001000500400304010100010040004000BD
:102350004000010140004000000202004000000275
:1023600040000102040440004000400040002120E1
:10237000B5C400000000000000000000D1C400004F
:102380000000000049A4000091AB000009B3000068
:10239000FF830000ADA0000000000000000000006E
:1023A000000000000000000000000000000000002D
:1023B000000000000000000000000000000000001D
:1023C000000000006BA300000000000000000000FF
:1023D0000600FF0901A101150026FF0075089540C0
:1023E0000901810295400901910295010901B1029B
:1023F000C00021006B0012011002EF020140280D05
:10240000040200100102030100000A0000000000A5
:102410000306AA00080002000400A0001400030044
:1024200057494E55534200000000000000000000D4
:102430008400040007002A0044006500760069005B
:102440006300650049006E0074006500720066005C
:1024500061006300650047005500490044007300B7
:10246000000050007B003900320043004500360078
:102470003400360032002D003900430037003700A9
:102480002D0034003600460045002D003900330091
:10249000330042002D003300310043004200390078
:1024A00043003500410041003300420039007D0007
:1024B00000000000050F3900021810050038B608AA
:1024C00034A909A0478BFDA0768815B665000121C7
:1024D000001C100500DF60DDD88945C74C9CD26523
:1024E0009D9E648A9F00000306AA00200009028BBB
:1024F0000005010080FA09040000020806500807E0
:1025000005820240000007050202400000080B019E
:10251000020202010409040100010202010405246F
:10252000001001052401030204240206052406010B
:10253000020705830310002009040200020A0000BC
:102540000507050402400000070584024000000959
:1025500004030002030000060921000100012221FA
:102560000007058103400001070501034000010940
:1025700004040000FF030007000000000403090436
:102580000803410052004D00300342004200430066
:1025900020006D006900630072006F003A00620065
:1025A00069007400200043004D00530049005300AF
:1025B0002D004400410050001A033000300030006C
:1025C0003100410030003000300030003000300079
:1025D000300022036D00620065006400200053009B
:1025E00065007200690061006C00200050006F00FF
:1025F0007200740022036D00620065006400200018
:10260000530065007200690061006C0020005000FA
:102610006F0072007400140343004D005300490022
:1026200053002D0044004100500024035700650072
:1026300062005500530042003A00200043004D0064
:102640005300490053002D00440041005000100386
:102650005500530042005F004D005300430000004E
:10266000000000000000000000BE0AE00D782D060A
:1026700068400824400000D35840641EFAD1491C29
:10268000521E002AF2D17047002070470020704788
:1026900070B5264C022060600120E060244D28685F
:1026A000C00702D00020606070BD00F02CF8F6E793
:1026B00070B51E4C022161601E49884202D3012080
:1026C000606100E0A0601A4D00F01DF82868C007A6
:1026D000FAD00020606070BDF8B505468E0813483A
:1026E000012114464160124F01CC01C53868C00772
:1026F00006D0761EF8D10D48002141600846F8BD8D
:1027000000F001F8F2E70C4840680006000E0BD01C
:102710000A494968002907D009490A4AC30700D075
:102720000A60091D4008F9D17047000000E501402A
:1027300000E40140001000100004014000050140C9
:10274000000601403546526E0000000021000020C6
:1027500025000020290000204900002071000020F1
:102760000000000001000020700100200010002087
:102770000002002000000020500100006826010037
:102780000002000068747470733A2F2F6D696372D1
:102790006F6269742E6F72672F6465766963652F47
:1027A0003F69643D404226763D405600393930301D
:1027B0000000000039393031000000000000000046
:1027C000496E206170706C69636174696F6E20700E
:1027D000726F6772616D6D696E6720736563746F88
:1027E00072206572617365206661696C65642E0094
:1027F000496E206170706C69636174696F6E2070DE
:10280000726F6772616D6D696E67206D61737320A1
:102810006572617365206661696C65642E000000F5
:10282000496E206170706C69636174696F6E2070AD
:10283000726F6772616D6D696E672077726974651A
:10284000206661696C65642E00000000496E20619D
:1028500070706C69636174696F6E2070726F6772FB
:10286000616D6D696E6720696E697469616C697A02
:102870006174696F6E206661696C65642E0000008A
:10288000496E206170706C69636174696F6E20704D
:10289000726F6772616D6D696E6720756E696E69C2
:1028A00074206661696C65642E00000054686520C0
:1028B0006865782066696C652063616E6E6F742050
:1028C00062652070726F6772616D6D65642E204C59
:1028D0006F676963206661696C757265206F6363F9
:1028E00075727265642E00005468652068657820F2
:1028F00066696C652063616E6E6F7420626520642A
:1029000065636F6465642E20506172736572206C1C
:102910006F676963206661696C757265206F6363B8
:1029200075727265642E00005468652068657820B1
:1029300066696C652063616E6E6F742062652064E9
:1029400065636F6465642E20436865636B73756DA2
:102950002063616C63756C6174696F6E2066616978
:102960006C757265206F636375727265642E00000A
:10297000546865206170706C69636174696F6E2062
:1029800066696C6520666F726D617420697320756D
:102990006E6B6E6F776E20616E642063616E6E6F1A
:1029A000742062652070617273656420616E642FAB
:1029B0006F722070726F6365737365642E00000020
:1029C000496E206170706C69636174696F6E20700C
:1029D000726F6772616D6D696E67206E6F742073C0
:1029E0007570706F72746564206F6E20746869739F
:1029F000206465766963652E00000000496E2061E1
:102A000070706C69636174696F6E2070726F677249
:102A1000616D6D696E67206661696C6564206265D1
:102A20006361757365207468652075706461746591
:102A30002073656E742077617320696E636F6D70AB
:102A40006C6574652E0000005468652073746172B3
:102A500074696E67206164647265737320666F7257
:102A60002074686520696E7465726661636520759F
:102A700070646174652069732077726F6E672E00D1
:102A8000546865207374617274696E672061646450
:102A90007265737320666F722074686520626F6F51
:102AA000746C6F616465722075706461746520690F
:102AB000732077726F6E672E0000000054686520E7
:102AC000626F6F746C6F616465722043524320645F
:102AD0006964206E6F7420706173732E00000000B3
:102AE000496E206170706C69636174696F6E2070EB
:102AF000726F6772616D6D696E672061626F72746B
:102B000065642064756520746F20616E206F757434
:102B1000206F6620626F756E6473206164647265F5
:102B200073732E00546865206865782066696C654B
:102B3000206F6666736574206C6F616420616464E5
:102B400072657373206973206E6F7420636F727285
:102B50006563742E00000000546865207472616E15
:102B6000736665722074696D6564206F75742E00DC
:102B700046696C652073656E74206F7574206F668E
:102B8000206F726465722062792050432E20546158
:102B900072676574206D69676874206E6F74206257
:102BA000652070726F6772616D6D656420636F720E
:102BB000726563746C792E00466C61736820616C79
:102BC000676F726974686D20777269746520636FCE
:102BD0006D6D616E64204641494C555245000000C0
:102BE000466C61736820616C676F726974686D20F0
:102BF000657261736520616C6C20636F6D6D616ED1
:102C000064204641494C555245000000466C6173B2
:102C10006820616C676F726974686D20657261739A
:102C20006520736563746F7220636F6D6D616E6490
:102C3000204641494C55524500000000546865202B
:102C40006865782066696C6520796F752064726F9D
:102C5000707065642069736E277420636F6D706196
:102C60007469626C65207769746820746869732080
:102C70006D6F6465206F72206465766963652E20D0
:102C800041726520796F7520696E204D41494E541F
:102C9000454E414E4345206D6F64653F2053656549
:102CA0002048454C50204641512E48544D000000CC
:102CB00054686520696E7465726661636520666933
:102CC000726D77617265204641494C454420746FAE
:102CD00020696E697469616C697A65207468652021
:102CE000746172676574204D435500005468652017
:102CF000696E74657266616365206669726D77617D
:102D00007265204641494C454420746F20646F77BA
:102D10006E6C6F61642074686520666C61736820F6
:102D200070726F6772616D6D696E6720616C676F3D
:102D3000726974686D7320746F20746865207461A3
:102D400072676574204D435500000000546865208B
:102D5000696E74657266616365206669726D77611C
:102D60007265204641494C454420746F207265735A
:102D700065742F68616C7420746865207461726773
:102D80006574204D43550000456E64206F662073C6
:102D9000747265616D20686173206265656E207272
:102DA000656163686564000054686520696E7465D8
:102DB0007266616365206669726D7761726520462F
:102DC00041494C454420746F20646F776E6C6F618D
:102DD000642074686520666C617368206461746146
:102DE00020636F6E74656E747320746F206265204B
:102DF00070726F6772616D6D65640000506F737300
:102E000069626C65206D69736D61746368206265C9
:102E1000747765656E2066696C652073697A6520D4
:102E2000616E642073697A652070726F6772616D7C
:102E30006D656400416E20696E7465726E616C2010
:102E40006572726F7220686173206F63637572724E
:102E500065640000416E206572726F722068617354
:102E6000206F6363757272656400000054686520AA
:102E7000696E74657266616365206669726D7761FB
:102E80007265204641494C454420746F20756E6C34
:102E90006F636B2074686520746172676574206667
:102EA0006F722070726F6772616D6D696E6700007E
:102EB0004F7065726174696F6E20776173207375EE
:102EC000636365737366756C00000000456E642073
:102ED0006F662073747265616D20697320756E6B07
:102EE0006E6F776E00000000416E206572726F7227
:102EF000206F6363757272656420647572696E67B2
:102F000020746865207472616E73666572000000DB
:102F100054686520696E74657266616365206669D0
:102F2000726D776172652041424F52544544207062
:102F3000726F6772616D6D696E672E20496D616792
:102F40006520697320747279696E6720746F2073CD
:102F5000657420736563757269747920626974732E
:102F6000000000004120626F6F746C6F61646572D5
:102F70002075706461746520776173207374617269
:102F80007465642062757420756E61626C6520746E
:102F90006F20636F6D706C6574652E0D0A52656CE1
:102FA0006F61642074686520626F6F746C6F616418
:102FB000657220746F206669782074686973206573
:102FC00072726F72206D6573736167652E0D0A00F2
:102FD000696E74657266616365000000696E746590
:102FE000726E616C00000000757365720000000075
:102FF00074617267657400007472616E7369656EE6
:10300000740000004D4245442020202056465320A5
:10301000202020202020202020202020302E3100A1
:103020004030010000F0FF1FA8020000A688000049
:10303000D4300100A8F2FF1F6830000004810000B6
:10304000041ABC2701180801010206020208012A1D
:1030500004052F010106060604017A1001051F016F
:103060009996970B1901016341237BCD23BDE11490
:103070004D1B0123A5C91A8D101AC51014491D0135
:103080001AAD100185176CDC0204300140292C03B5
:10309000016F732E6D6265642E636F6D2F776562AD
:1030A0007573622F6C616E64696E672D7061676500
:1030B0002F3F6269643DCA132C01211A5501012575
:1030C0003204AA010D11122012408D204C27011745
:1030D00001CF0000FFFFFFFFFFFFFFFFFFFFFFFF2C
:1030E000FFFFFFFFFFFFFFFFFFFFFFFFFFFFFFFFF0
:1030F000FFFFFFFFFFFFFFFFFFFFFFFFFFFFFFFFE0
:10310000FFFFFFFFFFFFFFFFFFFFFFFFFFFFFFFFCF
:10311000FFFFFFFFFFFFFFFFFFFFFFFFFFFFFFFFBF
:10FBF000FFFFFFFFFFFFFFFFFFFFFFFF127E2B3F17
:00000001FF
